:046F9C0001000146A9
:106A0D00AF50055074D02FF582E4341DF583E59910
:106A1D00F022D3E5309400E52F94002290000FE092
:036A2D00640322DD
:030003000257FFA2
:0B57FF00C0E0C083C082C0D075D0089D
:10580A00852E82852D83E493FF201404C4540FFF50
:10581A00430FF08F80C284D28500C2870000D287EE
:10582A00007580FF7580FEC284C28500C2870000B1
:10583A00D287007580FF30140CC214052EE52E7035
:09584A0006052D8002D214D2A83B
:09585300D0D0D082D083D0E03225
:03000B000219696E
:10196900C0E0C0F0C083C082C0D075D008758CD8E3
:10197900758A92D28C124228126350E531D39400B1
:1019890040171531E53164056009E531640F6003DD
:10199900021B7B126C52021B7B753114E54ED394EA
:1019A900004002154EE54FD394004002154FE53A29
:1019B900D394004002153AE54BD394004002154BED
:1019C900154CE54C123A5E1B6D001B42011B1A02B5
:1019D9001AF2031A6F041A56051A3D061A24071A31
:1019E9000B0819F20900001B78D3E52C9400E52BAC
:1019F90094005003021B7BE52C152C704D152B020E
:101A09001B7BD3E5379400E53694005003021B7B1A
:101A1900E537153770021536021B7BD3E54894006C
:101A2900E54794005003021B7BE5481548700215F1
:101A390047021B7BD3E54A9400E549940050030211
:101A49001B7BE54A154A70021549021B7BD3E52A1F
:101A59009400E52994005003021B7BE52A152A709E
:101A6900021529021B7B7885E6FF7003021B7BEFB9
:101A7900B40105900524801BEFB40210126A1F40BF
:101A89002FE53015307002152F021B7BEFB4030CC4
:101A9900900526E0F52FA3E0F5308028EFB4041275
:101AA900126A1F400BE53015307002152F021B7B9F
:101AB9008012EF64057003021B7BEFB4060C752FCF
:101AC90002753058788506021B7BEF6407600302B4
:101AD9001B7B126A1F400BE53015307002152F026F
:101AE9001B7B78857600021B7BD3E5399400E538AA
:101AF90094004008E539153970021538D3E53C944E
:101B090000E53B9400406BE53C153C7002153B80B9
:101B190061D3E5579400E55694004008E5571557F9
:101B290070021556D3E5559400E55494004043E5F9
:101B3900551555700215548039D3E5359400E534AF
:101B490094004008E535153570021534301523D356
:101B5900E5339400E53294004018E53315337012EB
:101B69001532800EE551D39400400415518000755B
:0D1B79004C0AD0D0D082D083D0F0D0E03222
:03001300023EF3B7
:0D3EF300C0E0C0F0C083C082C0D075D01008
:103F0000E545C394504003023FB7202403023FB766
:103F1000300C03023FB7E5A0540FF5587D077F0131
:103F2000124EE95067202364E545700DE558B40C46
:103F300008201105D211023FB720034A2011471271
:103F40003FC250047F0180027F0F126F1F90000F4D
:103F5000E0FF64016012EFB40302800C90000FE0F8
:103F6000B40209123FC250047F80801290000FE01B
:103F7000B4020E7D037F07124EE940057FA01200B8
:103F800016754202D20390053CE0F53A7D087F05A4
:103F9000124EE9502290002BE0B55807202304D29E
:103FA000268014053EE53EAE3D7002053D14F582C7
:073FB0008E83E558F0054582
:103FB700D0D0D082D083D0F0D0E0327D037F0712FB
:033FC7004EE9229E
:030023000264294B
:10642900C0E0C083C082C0D075D018309819C29816
:10643900E599B40A08126A0D755000800AE550C33F
:1064490094905003126A0D309902C299D0D0D0822B
:05645900D083D0E03209
:03003B0002493047
:0D493000C0E0C0F0C083C082C0D075D018B8
:10493D00C2CEE546C3941040030249C830257C2001
:10494D000C79AFA07804EF08800123D8FDF55953F9
:10495D00590F7D077F02124EE95035202332E5466F
:10496D00700CE559B40C07201304D213804D2004AC
:10497D001920131690000FE0B4020F7F0A126F1F5B
:10498D007F80120016754202D20490053CE0F53A84
:10499D007D087F05124EE9502290002BE0B5590796
:1049AD00202304D22880140540E540AE3F70020557
:0B49BD003F14F5828E83E559F005469B
:0B49C800D0D0D082D083D0F0D0E032FD
:104B9500E4F55AF55B755C1E755DFF855B82855A8C
:104BA50083E0F55E635EFFE55EF0E0655E6003123F
:104BB5006FA0635EFF855B82855A83E55EF0E065E5
:104BC5005E6003126FA0055BE55B7002055AE55D4B
:104BD500155D7002155CD3E55D9400E55C940050AD
:104BE500BA75985A758921758845758DE7758780D9
:104BF500758CD8758AEF75C90275C808753D1E751F
:104C05003E60753F1E7540B075B701D2A9D2E8D296
:0F4C1500AA75C64C75EEFF75FEFFD2AF12675839
:014C2400226D
:026FA00080FE71
:1069EA00202F0F90053AE0F54EE54ED39400401261
:1069FA0080F7302F0D90053AE0F54FE54FD394001C
:036A0A0050F9221E
:1069A20030310AD215900024E04420800DC2157FB8
:1069B20008126F60900024E054DFF0FD7F247E0017
:0469C2001263F32247
:102ECA008F70E570640170292030047F01805620DC
:102EDA003003022FC5122FD64003022FC5122FDE50
:102EEA00500C122FC6301503022FC5022FBB022F1A
:102EFA007BE570640270202030047F028027203036
:102F0A0003022FC5122FE64003022FC5126A297049
:102F1A0003022FC5022F95E57064036003022FC5D3
:102F2A002030057F03026F60303024122FD6501FE5
:102F3A00122FE6501A126A296015122FDE500B7FE3
:102F4A000B122FEE201574022FBB7F03022FC23003
:102F5A003023122FFC501E7D017F02124EE94015CC
:102F6A007D017F07124EE95008122FC620154C80AA
:102F7A00407F018043303017122FFC40127D017FC1
:102F8A0002124EE95009126A2960047F0280293030
:102F9A0030297D017F01124EE95020126A29701BE7
:102FAA007D017F07124EE9500D7F09122FEE201581
:102FBA000AD2310269A27F01126F73227F09126F4E
:102FCA0073900536E0F532A3E0F533227D017F01E7
:102FDA00124EE9227D017F07124EE9227D017F020E
:102FEA00124EE922126F73900536E0F532A3E0F52E
:0A2FFA0033227D017F01124EE9220F
:104C2500C2957FFF126F60124B957F071263875005
:104C35000512003E800312610ED28C7F0812638735
:104C450050051242E880FEC22B1268E89000D1E0C0
:104C5500FF7C117D00125C48125DBB90000FE0B433
:104C65000105122831801090000FE0FF64026004F6
:104C7500EFB40303123265123D32301E11E5427066
:104C85000DE52754A060077FA0126F1FC21E7D0788
:104C95007F05124EE94002C200E552C3940A50BB9B
:104CA5003015B8E533453270B2C2311269A280AB16
:104A6C00EF253EFFEE353DCF2401FDE43FFC22AFA8
:104A7C005A7E00EF2403FDEE33FC22E53E255AF569
:104A8C0082E4353DF58322E540255AF582E4353F35
:104A9C00F58322E56F256DF582E4356EF583E0FF35
:104AAC00E56F256DF582E4356EF58322E55A240217
:104ABC00FFE433FE22E56C2401FFE433FEC3E56D15
:104ACC009FEE6480F874809822EF2540FFEE353F0E
:104ADC0022C2017FF47E01126CC4E56C25E0F56CFA
:104AEC00756D0122E55C2EF582E4355BF583E0FD06
:084AFC0022753D1E753E60228B
:106CC400EF1FAA0670011ED39400EA9400400BE45F
:0A6CD400FDEDC394C850E90D80F7F0
:016CDE002293
:1051FE008F5BE55BB401197D017F06124EE9500C01
:10520E009000B1E0FF7C0D7D00125C48788506228F
:10521E00E55BB4021312527050439000B2E0FF7C73
:10522E000D7D20125C488035E55BB4041612527079
:10523E00500C9000B4E0FF7C0D7D60125C487885C8
:10524E00760622E55BB403197D027F06124EE95005
:10525E000C9000B3E0FF7C0D7D40125C48788576A3
:0A526E0001227D027F06124EE922A4
:104EE900BF0107900020E0FE8048BF020790002123
:104EF900E0FE803EBF0307900022E0FE8034BF043D
:104F090007900023E0FE802ABF0507900024E0FEF9
:104F19008020BF0607900025E0FE8016BF07079096
:104F29000026E0FE800CBF0807900027E0FE800203
:104F3900E4FEBD0103EE1322BD0204EEA2E122BD8F
:104F49000304EEA2E222BD0404EEA2E322BD05049D
:104F5900EEA2E422BD0604EEA2E522BD0704EEA2FC
:074F6900E622BD0802EE3351
:014F7000221E
:101D8700124AFD900100E0F55A124A87E0123A5EC6
:101D97001DB6011DEB021E20031E55041E8A051EDB
:101DA700BF061EF4071F24081F500900001F7A12E0
:101DB7004A87A3E0B40A15E55A124ABAE545B507BA
:101DC7000BE4B506077D017F01021F38124A7BE548
:101DD700456D7001EC6003021F7A124A6CC2297FBD
:101DE70001021F4D124A87A3E0B40A15E55A124AA9
:101DF700BAE545B5070BE4B506077D017F02021F6B
:101E070038124A7BE5456D7001EC6003021F7A12B8
:101E17004A6CC2297F02021F4D124A87A3E0B40A07
:101E270015E55A124ABAE545B5070BE4B506077D2D
:101E3700017F03021F38124A7BE5456D7001EC6094
:101E470003021F7A124A6CC2297F03021F4D124AEE
:101E570087A3E0B40A15E55A124ABAE545B5070B58
:101E6700E4B506077D017F04021F38124A7BE5456A
:101E77006D7001EC6003021F7A124A6CC2297F045D
:101E8700021F4D124A87A3E0B40A15E55A124ABA4F
:101E9700E545B5070BE4B506077D017F05021F3849
:101EA700124A7BE5456D7001EC6003021F7A124A06
:101EB7006CC2297F05021F4D124A87A3E0B40A1599
:101EC700E55A124ABAE545B5070BE4B506077D01A1
:101ED7007F06021F38124A7BE5456D7001EC6003EF
:101EE700021F7A124A6CC2297F06021F4D124A87C7
:101EF700A3E0B40A14E55A124ABAE545B5070AE45D
:101F0700B506067D017F078028124A7BE5456D707F
:101F170001EC705F124A6CC2297F078029124A8739
:101F2700A3E0B40A0F124A87A3A3E070077D017FDD
:101F370008024E5E124A7BE5456D7001EC70341263
:101F47004A6CC2297F08020FFB124A87A3A3E070DD
:101F570022124A87A3E024F96008147016E4FF02EE
:101F67005F987FF47E01126CC47D5E7F0212672E3C
:031F77001242E82B
:011F7A002244
:101B8600753F1E7540B0900108E0F55A124A93E081
:101B9600123A5E1BB8011BF0021C28031C60041CD1
:101BA60098051CD0061D08071D3B081D700900007E
:101BB6001D86124A93A3E0B40A13124AB8E546B545
:101BC600070BE4B506077D017F01021D53AF5A12CC
:101BD6004A7DE5466D7001EC6003021D86124AD50A
:101BE600124A73D2297F01021D6D124A93A3E0B4F3
:101BF6000A13124AB8E546B5070BE4B506077D0198
:101C06007F02021D53AF5A124A7DE5466D7001EC04
:101C16006003021D86124AD5124A73D2297F020238
:101C26001D6D124A93A3E0B40A13124AB8E546B5ED
:101C3600070BE4B506077D017F03021D53AF5A1259
:101C46004A7DE5466D7001EC6003021D86124AD599
:101C5600124A73D2297F03021D6D124A93A3E0B480
:101C66000A13124AB8E546B5070BE4B506077D0127
:101C76007F04021D53AF5A124A7DE5466D7001EC92
:101C86006003021D86124AD5124A73D2297F0402C6
:101C96001D6D124A93A3E0B40A13124AB8E546B57D
:101CA600070BE4B506077D017F05021D53AF5A12E7
:101CB6004A7DE5466D7001EC6003021D86124AD529
:101CC600124A73D2297F05021D6D124A93A3E0B40E
:101CD6000A13124AB8E546B5070BE4B506077D01B7
:101CE6007F06021D53AF5A124A7DE5466D7001EC20
:101CF6006003021D86124AD5124A73D2297F060254
:101D06001D6D124A93A3E0B40A12124AB8E546B50D
:101D1600070AE4B506067D017F078031AF5A124AED
:101D26007DE5466D7001EC7057124AD5124A73D2A2
:101D3600297F078032124A93A3E0B40A13124AB8E5
:101D4600E546B5070BE4B506077D017F08024E5E42
:101D5600AF5A124A7DE5466D7001EC7023124AD5E2
:101D6600124A73D2297F08020FFB124A93A3A3E0FB
:101D7600700E124A93A3E024F870057F01125F9853
:011D8600223A
:0447E3008C5B8D5C02
:1047E700055CE55C7002055B14F5828C83E0F9706B
:1047F7000302488AEF7005124AFD8009BF0106755A
:104807003F1E7540B0302946EF7007E965456002E5
:10481700C322BF0107E965466002C322E4FEEEC377
:10482700995029EF700F124AF0E53E2E124A8BE09D
:104837006D6002C322EF6401700F124AF0E5402E4B
:10484700124A97E06D6002C3220E80D2D32220293C
:1048570033E4FEEEC3995029EF700F124AF0E53E9C
:104867002E124A8BE06D6016C322EF6401700F129F
:104877004AF0E5402E124A97E06D6002C3220E808F
:04488700D2D322C3A3
:01488B00220A
:060FFB008F5BAB05AA04A8
:101001007D027F07124EE95011E55BB4050C8B821E
:101011008A83E0640570030212687D017F07124E26
:10102100E95011E55BB4050C8B828A83E06406709C
:1010310003021268C22AEB24FFF582EA34FFF5832A
:10104100E0F55D8B828A83E0FFF55EA3E0F9F55F51
:10105100EF123A5E107101107802107F03108604BE
:10106100108D05109406109B0710A208000010A710
:10107100755C01D22A802F755C02D22A8028755CAA
:1010810004D22A8021755C08D22A801A755C10D29C
:101091002A8013755C20D22A800C755C40D22A808C
:1010A10005755C80D22AE924FE700302116924F8D7
:1010B100605C2409600302117BE55BB401059000CB
:1010C100208045E55BB40205900021803BE55BB4DF
:1010D10003059000228031E55BB404059000238074
:1010E10027E55BB40505900024801DE55BB406058A
:1010F1009000258013E55BB407059000268009E583
:101101005B64087077900027E0455CF0806EE55BDA
:10111100B401059000208045E55BB40205900021F3
:10112100803BE55BB403059000228031E55BB404AC
:10113100059000238027E55BB40505900024801D00
:10114100E55BB406059000258013E55BB4070590C7
:1011510000268009E55B64087022900027E0FFE526
:101161005CF4FEEF5EF08014E55BB4050D8B828AC2
:1011710083E0FFD22F122992C22AC22A202A030217
:101181001268E55BB40109900020E0FD7F208060DA
:10119100E55BB40209900021E0FD7F218052E55B0F
:1011A100B40309900022E0FD7F228044E55BB40492
:1011B10009900023E0FD7F238036E55BB4050990AB
:1011C1000024E0FD7F248028E55BB406099000251A
:1011D100E0FD7F25801AE55BB40709900026E0FD5C
:1011E1007F26800CE55BB4080C900027E0FD7F278B
:1011F1007E001263F3126DBED2AF2029047F0180FD
:10120100027F02126F73A229922F1269EAAD5DE487
:10121100FF12672EAD5EE4FF12672EE55FB4010495
:101221007D388007E55FB40A077D367F0612672E99
:10123100E55BB4050312658B7D077F05124EE9500E
:101241000A200007C2307F03122ECA7D017F0112DE
:101251004EE94005C230122ECA7D017F02124EE9CD
:071261004005C230122ECA45
:011268002263
:024E5E008F5B68
:104E6000ED24FF922F1269EAE55B123A5E4E89014A
:104E70004E8E024E93034E98044E9D054EA2064E52
:104E8000A7074EAC0800004EB29000208021900091
:104E900021801C9000228017900023801290002413
:104EA000800D90002580089000268003900027E068
:104EB000F55CE55C6024755E01E4F55DE55C30E081
:104EC00007AD5EE4FF12672EE55CC313F55C055E7B
:104ED000055DE55DC3940840E3227D187F021267FB
:084EE0002E7D537F0212672EA4
:014EE80022A7
:10638700C2AFD284C285BF070BC28600E580A2E2F6
:10639700922A8019BF080BC28600E580A2E3922AE1
:1063A700800BBF0508C28600E58013922AD286D2E9
:0563B70085D2AFA22A0F
:0163BC0022BE
:1045CE00C229D22DE4FF125A757D2E7F0312672E5B
:1045DE007D607F0212672E7F03126F603024FD20F4
:1045EE0024FDE5456407703B7E017F50124AFD8F26
:1045FE00828E837407F07D01E53E2D124A8BE58293
:10460E0024FFF582E58334FFF583E0F9EF2DF58283
:10461E00E43EF583E9F00DBD08DED2297F647E000D
:10462E00126CC47F081263875043302995D22DE453
:10463E00FF125A757D607F0212672E7D327F061241
:10464E00672E7D1E7F0512672EC22DE4FF125A754E
:10465E007C017D507B087F507E011256777F0812B9
:10466E00638750097F327E00126CC480F07F647EB7
:04467E0000126CC4F6
:014682002215
:02560E008F5AB1
:10561000900138E0F55BE55A7020E55B124ABAE587
:10562000456F7001EE704F7460255BF582E4341EA7
:10563000AF82F55D8F5E7F408024E55A640170364D
:10564000E55B124ABAE5466F7001EE702974B02529
:105650005BF582E4341EAF82F55D8F5E7F10120031
:1056600016855E82855D83E0FFA3E0FD126E0C8FE0
:065670005CE4FD124F7125
:015676002211
:024F71008D6B46
:104F730075F020EF900280123A52AF8285836E8FD4
:104F83006FE0F56CD394004060E56C9410505AE5E3
:104F93006B7014124ADF124AC1504E124A9F124FCD
:104FA300F2056D056D80EFE56B64017019124ADD42
:104FB300124AC15034124A9F124FF2302402802900
:104FC300056D056D80EAE56B6402701D124ADD1202
:104FD3004AC15015124A9FA3E0FD1265BB3024035A
:0E4FE300024DD1056D056D80E67F50126F1FE7
:084FF10022A3E0FD1265BB22C2
:100D2E00855C82855B83A3A3E0FF855C82855B8304
:100D3E00A3222430F58274003EF583EDF0AF62EF0E
:100D4E003395E0FEE55F2FF582E55E3EF58322E505
:100D5E00822406F582E43583F583E0FF126DE7AD5C
:100D6E0007AF63EF3395E0FEEF22A3A3E0FFE55C50
:100D7E002404F582E4355BF583E022E55F2405F576
:100D8E0082E4355EF583E022E55F2405F582E435E5
:100D9E005EF583E0FFE55F2406F582E4355EF583BC
:100DAE00E0228E69F56AAF68EF3395E0FEE5662FB7
:100DBE00F582E5653EF583222455F582E4340AF585
:100DCE0083EFF0E56275F007A422AF60EF3395E094
:100DDE00FEE56175F008900158123A52E5822FF542
:100DEE0082E5833EF58322E5662405F582E43565CA
:100DFE00F583E022E55E75F007A42454F582E43411
:100E0E000AF58322A3A3A3E0FF8D828C83E58224BF
:100E1E0004F582E43583F583E022E55E75F007A4E0
:100E2E002451F582E4340AF5832224E0F582740A13
:100E3E003EF583E5822DF582E5833CF58322E55E62
:100E4E0075F007A42453F582E4340AF58322E55F96
:100E5E002405F582E4355EF583E0FFE55F2406F5B3
:100E6E0082E4355EF583E022E55E75F007A4245238
:100E7E00F582E4340AF58322749F2562F582E43408
:100E8E0000F58322746F2562F582E43400F5832227
:100E9E002450F582E4340AF58322ECFF3395E0FE0C
:100EAE00EF25E0FFEE33FE75F02022E5602405F518
:100EBE0082E4355FF58322D3EF6480948022AB0702
:100ECE00AA068B828A83A3A3A3E0FFEB2404F582F8
:100EDE00E43AF583E0FD228F828E83A3A3A3E02262
:100EEE00855F82855E83A3A322AB5DAD5AAF5CAEF8
:100EFE005B22FFE562FD3395E0FCE55F2DF582E5B3
:100F0E005E3CF5832233CE33CE92E022A2E0CE13A6
:100F1E00CE132275F00AA42DFDE5F03CFCE5662209
:100F2E00E5602405F582E4355FF583E022E5627520
:100F3E00F008900158023A52E55E75F007A4245568
:100F4E00F582E4340AF583E022AB5AAD5DAF5CAEB8
:100F5E005B22EF7C002563FDEC35628D82F58322EA
:100F6E00A3A3E0FFAD5A22540FF5657808AF03AE88
:100F7E0002EF08220564E564AE632275F020123A92
:100F8E0052E0FEA3E0FF22E0FAA3E0FB780CFFAEF6
:100F9E00020822E0FCA3E0FD7804FFAE040822E57F
:100FAE00632561F582E43562F58322E5662DF582CF
:100FBE00E5653CF58322E5662FF582E5653EF58312
:100FCE00222431F5827400222480F58274023EAF11
:100FDE0082222560F560E4355FF55F2285608285AB
:0D0FEE005F83228F828E83A3A3E0640A221A
:02055B008F5AB5
:10055D00C22AE4F542D223D22D125A757D4B7F0269
:10056D0012672E7D02E4FF12672E7D32E4FF1267C3
:10057D002E7D607F0212672E7D027F07124EE9509D
:10058D00057F04126F60900528E0F536A3E0F5377E
:10059D007F03126F60E55A7006A22492298009E547
:1005AD005AB40104A2259229E53745367005D22AA1
:1005BD00020A223029DFE55A7006A2249229800909
:1005CD00E55AB40104A22592292029EAE55A700BB7
:1005DD00755B1E755C6085455D800EE55AB401093D
:1005ED00755B1E755CB085465DE55DD3940050036B
:1005FD00020A1C855C82855B83E0640B6003020A42
:10060D0017A3E0FFB40A0AE55DB40205D22A020A77
:10061D001CEF6401701E120D38A3E0640A7015E51D
:10062D005D6405700F120D38120D78120A4D1231DE
:10063D0038020A1C120D38E0B40111120D38A3E076
:10064D00B40109120EF7121725020A1C120D38E01B
:10065D006401701E120D38A3E064027015E55D642F
:10066D0005700F120D38120D78120A4D1261FC0231
:10067D000A1C120D38E06401701D120D38A3E064E0
:10068D00037014E55DB4050F120D38120D78FDAB36
:10069D005A123A84020A1C120D38E0B4011D120DD3
:1006AD0038A3E0B40415E55DD39405400EAB5AAD07
:1006BD005CAC5BAF5D123004020A1C120D38E064B5
:1006CD0001701D120D38A3E064057014E55DB405CD
:1006DD000F120D38120D78FDAB5A125B67020A1C12
:1006ED00120D38E06401701D120D38A3E064067020
:1006FD0014E55DB4050F120D38120D78FDAB5A12CD
:10070D004D44020A1C120D38E0B4011D120D38A320
:10071D00E0B40715E55DD39405400EAB5AAD5CAC66
:10072D005BAF5D124683020A1C120D38E064017046
:10073D001D120D38A3E064087014E55DB4050F12A9
:10074D000D38120D78FDAB5A126236020A1C120DCD
:10075D0038E0B40215120D38A3E0B40A0DE55DB40E
:10076D000308AF5A1263BD020A1C120D38E0B40221
:10077D0016120D38A3E0B4010EE55DB40E09120E8C
:10078D00F9122D8E020A1C120D38E0B40216120D4C
:10079D0038A3E0B4020EE55DB40709120EF9125349
:1007AD006B020A1C120D38E0B40215120D38A3E0CD
:1007BD00B4090DE55DB40308AF5A1255A2020A1C27
:1007CD00120D38E064027019120D38A3E0B409114E
:1007DD00E55DB4040C120D38120F6E1267D4020AC7
:1007ED001C120D38E064037021120D38A3E0640A69
:1007FD007018E55D64057012120D38120D78FD123A
:10080D006E0CAD5A124738020A1C120D38E0640303
:10081D007029120D38A3E064017020E55DD39405B5
:10082D004019120D38120D78FD126E0C855A62ABFF
:10083D005DAD5CAC5B123E13020A1C120D38E06418
:10084D00037021120D38A3E064027018E55D640594
:10085D007012120D38120D78FD126E0CAD5A126019
:10086D0018020A1C120D38E0B40315120D38A3E05E
:10087D00B4030DE55DB40308AF5A126094020A1C6F
:10088D00120D38E0B40318120D38A3E0B40410E5CE
:10089D005DD394034009120F571249D3020A1C125B
:1008AD000D38E0B40315120D38A3E0B4050DE55D68
:1008BD00B40308AF5A126DFA020A1C120D38E0B4D7
:1008CD000316120D38A3E0B4060EE55DB40509124A
:1008DD000EF912690E020A1C120D38E0640370192C
:1008ED00120D38A3E0B40711E55DB4040C120D38F8
:1008FD00120F6E126C18020A1C120D38E0B403169A
:10090D00120D38A3E0B4080EE55DB40409120EF91A
:10091D00126933020A1C120D38E064057014E55D8E
:10092D00B4040F120D2EA3A3E0FDAB5A121F7B02D0
:10093D000A1C120D38E0B40516120D7CB40B10E52F
:10094D005DD394054009120F57123391020A1C1200
:10095D000D38E064067014E55DB4040F120D2EA37E
:10096D00A3E0FDAB5A12216D020A1C120D38E0B442
:10097D000616120D7CB40B10E55DD39405400912DB
:10098D000F571226A8020A1C120D38E06409701ABE
:10099D00120D38A3E0B40A12E55DB4040D120D3842
:1009AD00A3A3E0FF125E04020A1C120D38E06409D5
:1009BD007018120D38A3E0B40110E55DB4040B12EC
:1009CD000D38120F6E1263198045120D38E0B409FF
:1009DD0017120D38A3E0B4020FE55DD3940440085F
:1009ED00120EF71214D78027120D38E06409701A11
:1009FD00120D38A3E0B40310E55DB4040B120D38ED
:100A0D00120F6E125D7280078000AF5A126C352086
:100A1D002A030205A2C21ED22DAF5A125A757D604D
:100A2D007F0212672E7D327F0312672E7F03126FB6
:0F0A3D0060125E4C7FFF126F1FE47885F6C223B4
:080A4C0022FD126E0CAD5A22CE
:081725008E5E8F5F8D608B6109
:10172D00120EE5FFE55F2404120D8DFD1264C68FC8
:10173D006274E22562F562C394005003021926E536
:10174D006294144003021926E5616406701D120DA2
:10175D0089B4010C120DD1120E9E7401F0021922E2
:10176D00120DD1120E9EE4F0021922E561640E6095
:10177D0003021844E55F240C120D8DFFB40A14E525
:10178D005F240D120D8DB40A0A120DD1120E2EE426
:10179D00F08013E55F240D120D8DFD126C8C120D72
:1017AD00D1120E2EEFF0E55F240A120D8DFFB40A53
:1017BD0014E55F240B120D8DB40A0A120DD1120E11
:1017CD007CE4F08013E55F240B120D8DFD126C8C03
:1017DD00120DD1120E7CEFF0E55F2409120D8DFF75
:1017ED00640A6006EFD39409400A120DD1120E520D
:1017FD00E4F08010E55F2409120D8DFF120DD1125A
:10180D000E52EFF0120D89FFB40B15E55F24061291
:10181D000D8DB40B0B120DD1120E0874FFF0800854
:10182D00121952120E08EFF012192E120DC6120EC9
:10183D009E7401F0021922E561640A706E120DD1D9
:10184D00120E2EE4120DD0120E7CE4F0E55F240989
:10185D00120D8DFF640A6006EFD39409400A120D34
:10186D00D1120E52E4F08010E55F2409120D8DFFA8
:10187D00120DD1120E52EFF0120D89FFB40B15E5BA
:10188D005F2406120D8DB40B0B120DD1120E0874C0
:10189D00FFF08008121952120E08EFF012192E12D5
:1018AD000DC6120E9E7401F0021922E561640970D5
:1018BD0068120DD1120E2EE4120DD0120E7CE41210
:1018CD000DD0120E52E4F0120D89FFB40B15E55F29
:1018DD002406120D8DB40B0B120DD1120E0874FFD0
:1018ED00F08013E55F2406120D8DFD126C8C120D28
:1018FD00D1120E08EFF0E55F2407120D8DFFE55FA5
:10190D002408120D8DFD126C8C120DD1120DC61204
:10191D000E9E7401F0D22C8002C22CAF60126EF5B7
:10192D0022E55F2407F582E4355EF583E0FFE55F90
:10193D002408F582E4355EF583E0FD126C8CE562DA
:10194D0075F007A422E55F2406F582E4355EF58384
:0C195D00E0FD126C8CE56275F007A4221E
:103138008F5E8D5FE55ED3941D5003023244E55ED9
:1031480094324003023244D22DAF5F125A757D4645
:103158007F0712672EAF5E1235B874E2255EF55E02
:10316800120E2AE07021120E76E0701B120E4CE04F
:103178007015120E02E0700F120F46700A12325DBF
:103188007D537F0202323A12324CE55E75F007A495
:10319800120E9EE070047D3680027D387F0612672D
:1031A8002E12324C120E28E0FFD394014034EF94D3
:1031B80013502F7D097F0612672E120E28123254E3
:1031C8007FF47E01126CC47D0E7F0312672E7D355D
:1031D8007F0612672E7D097F0612672E120E761261
:1031E80032547FF47E01126CC4120E4CE0FF60056D
:1031F800125B18800A12325D7D0F7F0312672E7DE5
:10320800277F0212672E120E02E0FFF46008126D8B
:10321800491235B880077D187F0212672E7D377FE7
:103228000412672E120F46FF126D491235B87D053C
:103238007F0612672EC22DAF5F025A75C22CAF5F90
:10324800126EF5227FF47E01126CC422E0FF126D2B
:0D325800491235B8227D187F0212672E2220
:0261FC008D5EB6
:1061FE00EFD3941D402AEF9432502574E22FFFE422
:10620E00FEEEFD3395E0FCEF75F007A42450F58209
:10621E00E4340A120E3FE4F00EBE07E5D22C8002E3
:07622E00C22CAF5E126EF5F9
:016235002246
:062D8E008E5E8F5F8D6078
:102D9400D22B120EE5FFE55F2404120DA7122EB507
:102DA400C39418501C855F82855E83A3A3A3E0FFB0
:102DB400E55F2404120DA7FD126DD47883A6078065
:102DC40006E47883F6C22B120D96122EB5C3943CFA
:102DD400500D120D96FD126DD47884A6078006E47A
:102DE4007884F6C22BE55F2407120DA7FF126E87C5
:102DF4008F61E561D394004017E56194085011E5B3
:102E04005F2407120DA7FF126E877880A60780063D
:102E140078807601C22BE55F2408120DA7FFE55FD9
:102E24002409120DA7122EBE401FE56194205019EB
:102E3400E55F2408120DA7FFE55F2409120DA7FD25
:102E4400126DD47888A607800678887601C22BE5AF
:102E54005F240A120DA7FFE55F240B120DA7122EA3
:102E6400BE401FE561940D5019E55F240A120DA7B9
:102E7400FFE55F240B120DA7FD126DD47881A60720
:102E8400800678817601C22BE55F240C120DA7FF22
:102E9400E55F240D120DA7FD126DD47882A60730CC
:102EA4002B07125914D22C8002C22CAF60126EF57B
:102EB40022FD1264C68F61E56122FD1264C68F6132
:062EC400E561D394002239
:06536B008E5E8F5F8D6075
:10537100D22B120EE5FFE55F2404120E6D1253D6F7
:105381009418501C855F82855E83A3A3A3E0FFE58B
:105391005F2404120E6DFD126DD47883A60780067A
:1053A100E47883F6C22B120E5C1253D6943C500D56
:1053B100120E5CFD126DD47884A6078006E4788411
:1053C100F6C22B302B07125914D22C8002C22CAFFB
:0453D10060126EF503
:0B53D50022FD1264C68F61E561C32257
:106E8700120EC54008EF6480948A5001227F0022C9
:106DD400AE05126E87EFC454F0FDAF06126E87EF56
:036DE4004DFF223E
:1063BD008F5ED22D125A757D1E7F0812672E7D2697
:1063CD007F0812672E7D527F0412672EC22B126832
:1063DD00E8125CDE7880E6FF125B18125A1FC22DA0
:0663ED00AF5E125A75229A
:1067D4008D5EEFD3940A4006EFD3940F4003EF701D
:1067E4000E90002BEFF0D22CAF5E126EF5D322C2C6
:0867F4002CAF5E126EF5C3220A
:0255A2008F5E1A
:1055A400D22D125A757D207F0512672E7D2E7F0322
:1055B40012672E7D527F0412672E90002BE0F55F58
:1055C400E55FB40B067D5F7F078034E55FB40C06AE
:1055D4007D5E7F068029E55FB40D067D0A7F02802B
:1055E4001EE55FB40E067D327F028013E55FB40FC3
:1055F400067D467F028008E55F70077D0A7F0312FF
:09560400672EC22DAF5E125A752B
:01560D00227A
:106C18008D5E120EC5400EEF648094865007126494
:0D6C28005ED22C8002C22CAF5E126EF522EF
:02690E008D5E9C
:10691000120ECC1264C6120EC54010EF648094A112
:106920005009900029EFF0D22C8002C22CAF5E12E9
:026930006EF502
:016932002242
:026933008D5E77
:10693500120ECC1264C6120EC54010EF648094A1ED
:106945005009900028EFF0D22C8002C22CAF5E12C5
:026955006EF5DD
:01695700221D
:106DE700D3EF648094814008EF6480948A50012235
:036DF7007F0022F8
:106E9700120EC54008EF648094A15001227F0022A2
:0814D7008E5E8F5F8D608B615A
:1014DF00120EE514F56374FC2561F5616403600F6A
:1014EF00E56164076009E561640B60030216C2C31E
:1014FF00E5636480948050030216C2E563648094B0
:10150F008840030216C2E4F562120D6F7803C333ED
:10151F00CE33CED8F92430F58274003EF583AF6216
:10152F00EF3395E0FE120DEAE4F00562E562B408D0
:10153F00D8756204E56164037029120D4B12170808
:10154F00120D6D7803C333CE33CED8F9120D40A3ED
:10155F00A3120D687803C333CE33CED8F9120FCF51
:10156F000216B9E56164077069120D4B1217081264
:10157F000D6D7803C333CE33CED8F9120D40A3A32C
:10158F00120D687803C333CE33CED8F9120FCF12B2
:10159F000D46A3A3A3120D687803C333CE33CED861
:1015AF00F92432F5827400120D461216CAC333CED7
:1015BF0033CED8F92433F5827400120D46120D5D27
:1015CF007803C333CE33CED8F92434F582740002B6
:1015DF0016B9E561640B60030216C2120D4BE012DF
:1015EF000F00A3E0FD1264C6126E97120D6D780303
:1015FF00C333CE33CED8F9120D40A3A3120D6878A2
:10160F0003C333CE33CED8F9120FCF120D46A3A397
:10161F00A3120D687803C333CE33CED8F92432F535
:10162F00827400120D461216CAC333CE33CED8F9C8
:10163F002433F5827400120D46120D5D7803C33307
:10164F00CE33CED8F92434F5827400120D46E582DC
:10165F002407120D617803C333CE33CED8F9243566
:10166F00F5827400120D46E5822408120E1F120F28
:10167F0000E5822409120E1FFD1264C6126E971226
:10168F000D6D7803C333CE33CED8F92436F582747B
:10169F0000120D46E582240A120D617803C333CE82
:1016AF0033CED8F92437F58274003EF583EDF0D2AE
:0A16BF002C8002C22CAF60126EF501
:1016C90022E5822404F582E43583F583E0FFE562AF
:1016D900FD3395E0FCE55F2DF582E55E3CF583E59C
:1016E900822405F582E43583F583E0FD1264C61290
:1016F9006E97AD07AF63EF3395E0FEEF780322E015
:10170900FFE562FD3395E0FCE55F2DF582E55E3C82
:0C171900F583A3E0FD1264C6126E972257
:045D72008D5EAC078F
:105D7600D3EC648094804035EC64809489502EE4A2
:105D8600FDECFF3395E0FEEF7803C333CE33CED878
:105D9600F92428F58274003EF583EDFF3395E0FE85
:105DA600120DEAE4F00DBD08D8D22C8002C22CAF49
:045DB6005E126EF516
:015DBA0022C6
:106319008D5E120EC5402FEF648094895028EF14CA
:10632900FFE55E24FF922B124FF9D22DAF5E125A70
:10633900757542017F327E00126CC4E54270FCC261
:076349002DAF5E125A752210
:084683008F5E8C5F8D608B617E
:10468B00856082855F83120E12FD1264C68F62E510
:10469B0062D394005003024730E562943240030228
:1046AB004730E55E64067036D22DAF61125A757DC8
:1046BB00527F0512672EAF621235B8120F2EB4015E
:1046CB000A120E867401F07D388007120E86E4F014
:1046DB007D367F0612672EC22DAF61025A75E560DB
:1046EB002406120F32640B703C120F2EB401081209
:1046FB000E867401F08005120E86E4F074F9255EC7
:10470B00F55E75F004123998AFF0EF7014E5602484
:10471B0006FBE4355FFAAD62E4FF1234B8D22C80AD
:0C472B0006C22C8002C22CAF61126EF599
:01473700225F
:083004008F5E8C5F8D608B6113
:10300C00856082855F83120E12FD1264C68F62E5A5
:10301C0062D394005003023130E5629428400302DD
:10302C003130E55E64067037D22DAF61125A757D72
:10303C00527F0512672EAF621235B8120EB9E0B48A
:10304C00010A120E927401F07D388007120E92E480
:10305C00F07D367F0612672EC22DAF61025A75E5E0
:10306C00602406120EBDE0640B6003023130120EB8
:10307C00B9E0B40108120E927401F08005120E92A0
:10308C00E4F0E4FFFEE5602407120EBDE5822E128B
:10309C000E1FB40B04AF0680040EBE08E8EF7003DD
:1030AC00023130C39408507C120F3BEFF07E01EFDD
:1030BC002401FDE433FCEEC39DEC6480F87480982D
:1030CC005020E5602406120EBDE5822E120E1FFD67
:1030DC00120F3BE5822EF582E43583F583EDF00E7D
:1030EC0080CDE5602408120EBDE5822F120E1F6400
:1030FC000B602DEF2408FEC3E55E9EF55E75F004B3
:10310C00123998AEF0EE701CE5602407FDE4355FD3
:10311C00FC7E00ED2FFBEE3CFAAD627F011234B861
:0B312C00D22C8002C22CAF61126EF5A5
:013137002275
:0834B8008F638D648A658B6649
:1034C000756801E4F567120DB4E0FF6409703E12FF
:1034D00035A98003120F13D8FB120DB012359B785B
:1034E00008EF088003120F13D8FB120DB0A3A3E05E
:1034F000FFE568FD3395E0FCE5662DF582E5653C6A
:10350000F583A3A3A3E0FD126E0C023554120DB493
:10351000E0FF1235A98003120F13D8FB120DB01271
:10352000359B7804EF088003120F13D8FB120DB0FF
:10353000A3A3E0FF126F56EF426AAE69AF6A780448
:10354000EF088003120F13D8FB120DB0A3A3A3E062
:10355000FF126F56EF426AE563700FAF67120D718D
:10356000120EAFE564900AC08012E563B40117AF94
:1035700067120D71120EAFE564900530120DE7E58C
:1035800069F0A3E56AF074042568F5680567C3E58A
:0A359000676480949050030234C673
:10359A0022A3E0FF126F56EF426AAE69AF6A2212A7
:0E35AA006F567569008F6AAE697804EF0822CB
:0A6F5600EFD3940940037F002222CC
:023A84008B5E57
:103A86001264C68F61E561D394005003023B66E57C
:103A96006194334003023B66D22DAF5E125A757DA8
:103AA600527F0512672EAF611235B8746F25611209
:103AB6000E96E060047D3880027D367F0612672E02
:103AC6007F2C7E01126CC4E561120F3DE0F55F703C
:103AD600077D1B7F0612672E7D577F0212672EE534
:103AE6005F603B756001AF5F120D712401FFE43E1C
:103AF600FEAD60ED3395E0FCC3ED9FEE6480F8EC1F
:103B06006480985019120DD8E0B40A04E4FD8006CA
:103B1600120DD8E0FDE4FF12672E056080C87F2CE9
:103B26007E01126CC4E561900530120F8990000089
:103B3600EEF0A3EFF04E70077D1B7F0612672E7D19
:103B46000C7F0312672E900000E07002A3E060096C
:103B5600E56114FD7F01122AF0C22DAF5E025A758F
:073B6600C22CAF5E126EF5E8
:013B6D002235
:024D44008B5E84
:104D46001264C68F5FE55FD394004077E55F9433C6
:104D56005071D22DAF5E125A757D527F0512672EA5
:104D6600AF5F1235B8749F255F120E8AE060047D2E
:104D76003880027D367F0612672E7F2C7E01126CEC
:104D8600C47F2C7E01126CC4E55F900AC0120F89A5
:104D9600900000EEF0A3EFF04E70077D1B7F061229
:104DA600672E7D0C7F0312672E900000E07002A331
:104DB600E06009E55F14FDE4FF122AF0C22DAF5E44
:0A4DC600025A75C22CAF5E126EF5A2
:014DD00022C0
:026236008B5E7D
:106238001264C6AD07EDD394004025ED9433502089
:10624800E4FC120EA8ED900AC0120DE7E4F0A3F0EA
:106258000CBC10EE749F2D120E8AE4F0D22C800232
:07626800C22CAF5E126EF5BF
:01626F00220C
:025B67008B5E53
:105B69001264C6AD07EDD394004036ED943350313D
:105B7900E4FC120EA8ED900530120DE7E4F0A3F055
:105B89000CBC10EE746F2D120E96E4F0FCECFF3392
:105B990095E0FEED120DE1E4F00CBC08F0D22C808A
:085BA90002C22CAF5E126EF582
:015BB10022D1
:042AF0008F628D6301
:102AF400E4F564E5627052AF64120D7125E0FDEEF9
:102B040033FCAF63120D717805C333CE33CED8F9DD
:102B1400120E38120F958003120F1AD8FB120F757C
:102B24008003120F1AD8FB540FF566AF63120D71B0
:102B34007805C333CE33CED8F9120E38120FA180E4
:102B440003120F1AD8FB022BAEE56264017064AF66
:102B540064120D7125E0FDEE33FCAF63120D717844
:102B640005C333CE33CED8F92450F5827405120E42
:102B74003E120F958003120F1AD8FB120F758003B3
:102B8400120F1AD8FB540FF566AF63120D71780556
:102B9400C333CE33CED8F92450F5827405120E3ED9
:102BA400120FA18003120F1AD8FB540FF567ED54CE
:102BB4000FF568E565700CE5667008E5677004E577
:102BC40068607CAD65E4FF12672EAD66E4FF1267B2
:102BD4002EE56564097045856769AF69FE7804EF81
:102BE400088003120F13D8FBF569E5684269E569AB
:102BF400B4990B7D09E4FF12672E7D098027E569EE
:102C040075F00A84F56AFDE4FF12672EE56A75F033
:102C14000AA4FFC3E5699FF56AFD8009AD67E4FF77
:102C240012672EAD68E4FF12672E7FF47E01126CEA
:0F2C3400C40564C3E564648094A05003022AF7CA
:012C4300226E
:1064C600EFD394004015EF940B5010EFC3940A508D
:1064D60008EF75F00AA4FE8002E4FEEDD3940040B6
:1064E6000EED940B5009EDC3940A5003ED2EFEAF4A
:0164F600069F
:0164F7002282
:0649D3008E5E8F5F8B6019
:1049D900756105756240D3ED64809484407CED6413
:1049E9008094A55075ED24FDF563D39404406BE5DF
:1049F9006320E06613F5640562E562AE6170020545
:104A09006114F5828E83E564F07403255FF55FE434
:104A1900355EF55EE4F563E563C395645033855F00
:104A290082855E83E0FFA3E0FD126E0C0562E562FC
:104A3900AC617002056114F5828C83EFF0055FE5C6
:104A49005F7002055E055FE55F7002055E056380C4
:104A5900C6D22CAF60126EF5D322C22CAF60126E93
:024A6900F5C393
:014A6B002228
:043E13008C5F8D60D3
:103E1700120EC55003023EEBEF64809495400302F7
:103E27003EEBEB648094875003023EEBEB64809497
:103E3700E44003023EEB120D717805C333CE33CE57
:103E4700D8F9120FD6F5638F64EB24FBF565D3948D
:103E5700025003023EEBE56575F00384E5F060036D
:103E6700023EEBE56575F00384F567C39410507463
:103E7700120F827002056314F5828E83E567F07472
:103E870005120FE0E4F565E565C395675052120F1B
:103E9700EAE0F566B40A10120F827002056314F5A2
:103EA700828E83E4F0800F120F827002056314F58F
:103EB700828E83E566F0120FEAA3E0FF120FEAA3F2
:103EC700A3E0FD126E0C8F66120F82700205631459
:103ED700F5828E83E566F07403120FE0056580A70F
:0B3EE700D22C8002C22CAF62126EF5DC
:013EF20022AD
:0826A8008E5E8F5F8D608B6177
:1026B000C22B120FF160030227451228205003029B
:1026C0002740E5649408E56394075074C3E56064AB
:1026D00080948A506B120EEEA3E0F562B40106906E
:1026E0000520022795E562B402069005220227958F
:1026F000E562B40306900524022795E562B404065A
:10270000900526022795E562B40506900528022764
:1027100095E562B4060690052A022795E562B4079E
:102720000690052C022795E562B4080590052E80D9
:1027300064E562B40905900530805AD22B02281155
:10274000D22B022811120EEEE064017052AD60AF80
:102750005FAE5E1228205003022811E5649408E55C
:102760006394074003022811C3E5606480948A40A3
:1027700003022811120EEEA3E0F562B40A059005DB
:10278000328012E562B401059005348008E562B438
:102790000209900536E563F0A3806FD22B80721298
:1027A0000EEEE06402706AAD60AF5FAE5E125BB2C7
:1027B0007563008F64C3E5649463E56394005051CE
:1027C000C3E560648094885048120EEEA3E0F56281
:1027D000B40107900538EFF08037E562B402059048
:1027E00005398026E562B4030590053A801CE56250
:1027F000B4040590053B8012E562B4050590053CE4
:102800008008E562B4060890053DE564F08002D2D8
:0F2810002B302B04C22C8002D22CAF61126EF53C
:10281F002212488C8E638F64D3E564943BE56394F6
:02282F00002285
:06488C008E658F66A90590
:104892007D057C00120FB9E0C3940A4005120FB9DE
:1048A200E4F00DBD00010CED640A4C70E7B9060797
:1048B200120DF5FF7E0022E964077010120DF575E6
:1048C200F00AA4ACF0FDE5662406801BE9640870DA
:1048D20021120DF575F064A4ACF0FDE56624061214
:1048E2000DF9120F212407120DF92DFDE43CAF053D
:1048F200FE22E964097033120DF5FF7E007C037D10
:10490200E81239BAAC06AD07E5662406120DF97550
:10491200F064120F242407120DF9120F2124081239
:0D4922000DF92DFDE43CFEAF0522E4FEFF83
:01492F002265
:065BB2008E658F66A90557
:105BB8007F057E00120FC4E0C3940A4005120FC48B
:105BC800E4F00FBF00010EEF64084E70E7E96407C8
:105BD8007020E5662405F582E43565F583E075F007
:105BE8000AA4FFE5662406F582E43565F583E02F0F
:045BF800FF227F0009
:015BFC002286
:083391008E5E8F5F8D608B6181
:10339900C22BD3E56064809484500302343FE56016
:1033A9006480948D400302343F120FF160030234AC
:1033B9003F120EE5123A5E33DF0133EA0233F503B9
:1033C90033FF04340905341306341D073427083440
:1033D90031090000343B756201756300D22B023458
:1033E90076756201756308D22B02347675620175B0
:1033F9006310D22B8077756201756318D22B806DAB
:10340900756201756320D22B80637562017563282B
:10341900D22B8059756201756330D22B804F75624A
:1034290001756338D22B8045756201756340D22BD3
:10343900803BC22B8037D3E56064809484402EE5BD
:10344900606480948D5026855F82855E83A3A3E0A6
:10345900B4011A855F82855E83A3A3A3E024F67075
:103469000A756201756358D22B8002C22B302B3743
:10347900E4FF120F60E4F00FBF08F7E56024FB8555
:103489006382856283F07F01E55F2404F582E43578
:103499005EF583E5822F120E1FFE120F60EEF00F0C
:0E34A900BF08E5D22C8002C22CAF61126EF576
:0134B70022F2
:044738008F5E8D5FA4
:10473C00E55ED3940050030247DBE55E941540031D
:10474C000247DBD22DAF5F125A757D5F7F05126772
:10475C002EAD5EE4FF12672E7D527F0412672E7F12
:10476C00F47E01126CC475F020E55E900280123A62
:10477C0052AF828583628F63E0F560603DD3940015
:10478C004046E56094105040E56025E0F5607561A9
:10479C0001E5602401FFE433FEC3E5619FEE648014
:1047AC00F87480985022120FADE0FF120FADA3E009
:1047BC00FD1265BB0561056180D77D1B7F06126705
:1047CC002E7D5F7F0512672EC22DAF5F025A75C218
:0647DC002CAF5F126EF528
:0147E20022B4
:10216D008F5E8D5F8B60E55E640A7074E55FC3946E
:10217D000A40030222DA122310E4FDFF12672EAD8E
:10218D005F1222E9E55F123A5E21B50121BB022102
:10219D00C10321C70421CD0521D30621D90721DF94
:1021AD000821E509000021EA90052002223490055E
:1021BD002202223490052402223490052602223474
:1021CD0090052802223490052A02223490052C0213
:1021DD00223490052E022234900530804A0222D3FB
:1021ED00E55E64017052E55FD394004006E55F94AF
:1021FD00034006E55F640A703C122310E55FB40AE4
:10220D000A7D0A1222E9900532801CE55FB4010AAD
:10221D007D0B1222F6900534800DE55FB402137D1F
:10222D000C1222F6900536E0FEA3E0FF12652A029D
:10223D0022E10222D30222DAE55E64026003022269
:10224D00E1E55FD3940050030222DAE55F94075075
:10225D007CD22DAF60125A757D277F0812672E7DB7
:10226D0006E4FF12672E7D14E4FF12672EE55F244E
:10227D00FE601A14602114602814602F1460362437
:10228D000570437D0112230390053880307D0212C5
:10229D00230390053980267D0312232690053A806D
:1022AD001C7D0412232690053B80127D05122333DD
:1022BD0090053C80087D0612233390053DE0FF7E9E
:1022CD000012655B800EAF60126C358007C22CAFBB
:1022DD0060126EF5C22DAF60125A7522E4FF1267BF
:1022ED002E7D527F0412672E22E4FF12672E7D523F
:1022FD007F0412672E22E4FF12672E7D527F041297
:10230D00672E22D22DAF60125A757D277F08126776
:10231D002E7D06E4FF12672E22E4FF12672E7D52FA
:10232D007F0412672E22E4FF12672E7D527F041266
:03233D00672E22E6
:044B04008E638F64C9
:104B08000564E5647002056314F5828E83E0F5663A
:104B1800607AC3940850757F2C7E01126CC4E4F54A
:104B280065E565C395665064856482856383E01294
:104B38003A5E4B75004B530A4B570B4B5D0C4B635E
:104B48000D4B690E4B6F0F00004B7BE4FD802D7DF4
:104B58005F7F0780287D5E7F0680227D0A7F028036
:104B68001C7D327F0280167D467F0280107D0A7F81
:104B780003800A856482856383E0FDE4FF12672E63
:0C4B88000564E564700205630565809516
:014B940022FE
:061F7B008F5E8D5F8B609C
:101F8100C22BE55E640A600302206FE55F123A5ED0
:101F91001FB0011FC3021FD6031FE9041FFC052048
:101FA1001206202807203E082053090000206B124A
:101FB10020A47D011220F2756101756200D22B020D
:101FC100208B1220A47D021220F275610175620836
:101FD100D22B02208B1220C07D031220FF756101DC
:101FE100756210D22B02208B1220C07D041220FFBB
:101FF100756101756218D22B02208B1220DC12212F
:10200100527D05122122756101756220D22B0220B9
:102011008B1220DC1221527D06122122756101757D
:102021006228D22B02208B12210C1221667D07120D
:10203100212F756101756230D22B02208B12210C88
:102041001221667D0812212F756101756238D22B2C
:10205100803812213CE4FDFF12672E7D09122159BF
:10206100756101756240D22B8020C22B801CE55E18
:1020710064017016E55F24F6701012213C7D0A128E
:102081002159756101756258D22B302B09AF62AEAF
:1020910061124B048005AF60126C35C22DAF601226
:0220A1005A756E
:1020A30022D22DAF60125A757D577F0212672E7DA3
:1020B30005E4FF12672EE4FDFF12672E22D22DAF37
:1020C30060125A757D577F0212672E7D05E4FF1259
:1020D300672EE4FDFF12672E22D22DAF60125A75D0
:1020E3007D577F0212672E7D05E4FF12672E22E4DF
:1020F300FF12672E7D527F0412672E22E4FF1267C0
:102103002E7D527F0412672E22D22DAF60125A7594
:102113007D577F0212672E7D05E4FF12672E22E4AE
:10212300FF12672E7D527F0412672E22E4FF12678F
:102133002E7D527F0412672E22D22DAF60125A7564
:102143007D577F0212672E7D05E4FF12672E22E47E
:10215300FDFF12672E22E4FF12672E7D527F0412C9
:0A216300672E22E4FDFF12672E2212
:1035B8008F72E572D3945940107D5A12369F24A613
:1035C800FD700302369E023699E572D3944F401679
:1035D800E572945A50107D5012369F24B0FD700346
:1035E80002369E023699E572D394454016E57294E8
:1035F8005050107D461236A724BAFD700302369E3D
:10360800023699E572D3943B4012E5729446500C09
:103618007D3C1236A724C4FD607C8075E572D39486
:10362800314012E572943C500C7D321236AF24CEF4
:10363800FD6063805CE572D394274012E572943292
:10364800500C7D281236AF24D8FD604A8043E572BD
:10365800D3941D4016E572942850107D1EE4FF1285
:10366800672EE57224E2FD602D8026E572D394135F
:103678004016E572941E50107D14E4FF12672EE583
:103688007224ECFD60108009E572C394145007ADF4
:1036980072E4FF12672E22E4FF12672EE57222E41D
:0F36A800FF12672EE57222E4FF12672EE57222F1
:105A75008F6AE56A700C302D097F01126F737FC044
:105A8500801FE56A700C202D097F01126F607FC0B1
:105A95008026E56AB40112302D0F7F02126F737FE5
:105AA50030120016C22F0269EAE56AB40114202DEE
:105AB500117F02126F607F30126F1F7FC87E001248
:035AC5006CC4228C
:1069C6008F69D22D125A757D607F0212672E7D3235
:1069D6007F0612672E7D1E7F0512672EC22DAF69B8
:0469E600125A7522AA
:106C35008F69D22D125A757D607F0212672E7D30C5
:0D6C45007F0312672EC22DAF69125A75220F
:0E6EF5008F68302C030269C6AF68126C35221C
:105E0400EF24FE60101460162402701C7F01126FD0
:105E1400737F8080107F02126F737F2080077F035F
:105E2400126F737FA01200167FF47E01126CC4758A
:105E34004204E54270FC7F647E00126CC47F03124E
:085E44006F607FA0126F1F22A6
:10655B008E618F627C007D0A1239CCAD07E4FF128D
:10656B00672E7D5B7F0612672EAE61AF627C007D6E
:10657B000A1239CCE4FF12672E7D4A7F0702672E81
:04652A008E618F628D
:10652E007C007D3C1239CC1235B87D057F06126792
:10653E002EAE61AF627C007D3C1239CCED4C600C0E
:0C654E00AF051235B87D4A7F0712672E9A
:01655A00221E
:026018008D5E9B
:10601A00120EC5402FEF648094955028120D7178A6
:10602A0005C333CE33CED8F9120FD6FEE4FD0FEFF7
:10603A00AA0670010E14F5828A83E4F00DBD20EEE3
:0B604A00D22C8002C22CAF5E126EF55B
:016055002228
:106094008F5E900540E0D394024015D22D125A75BC
:1060A4007542037F327E00126CC4E54270FC801599
:1060B400D22DAF5E125A757D1B7F0612672E7D0CA2
:0D60C4007F0312672EC22DAF5E125A7522A7
:106DFA007E10900540E4F0A3DEFC7E10D22C126EC9
:016E0A00F592
:016E0B002264
:106E0C00BF0A02E4FFBD0A02E4FDEF75F00AA42DEF
:026E1C00FF2253
:106C8C00EFD394094002E4FFEDD394094002E4FDF4
:0C6C9C007804EF08800123D8FD4DFF2292
:10409D0007010203040506070707060504030201CD
:1040AD0003010A0A030307050303020503020A0AB3
:1040BD0004050A0A0104050A0A0A04050A0A02038C
:1040CD00070A0A03040A0A04024B00020032072EF3
:1040DD0003024B0002003202055F000302055F0080
:1040ED000402055F000502055F000604072E082681
:1040FD000640033204072E08260640025304081E0C
:10410D0008260452010008024B00020032072E0857
:10411D001E08260452010003072B0235063603073D
:10412D002B0235063803072B0235072603072B0212
:10413D0035025302055F000F02055F001002055F97
:10414D00001102055F001202055F001302055F00FA
:0A415D0014080C0A1D020500241BC3
:1052F2007461F0A37420F0A37452F0A37401F0A3BC
:1053020022A3F0A37461F0A37440F022F0A374030B
:10531200F0E4A3F0A37410F0A37403F0E4A3F0A3E9
:10532200227461F0A37441F0A3227461F0A3F0A38C
:105332007430F0A3227496F0A37432F0A37495F043
:10534200A3741EF0A322F0A37461F0A314F0A3745B
:1053520070F0A3E4F022A3F0A37452F0A3223CF570
:0953620083E0FEEF3395E0FC222C
:10003E007E407F9D7C017D507B08125F167E407F47
:10004E00A57C017D587B08125F167E407FAD7C013A
:10005E007D007B04125F167E407FB97C017D087B9C
:10006E0004125F167E407FB57C017D107B04125F0B
:10007E00167E407FB17C017D187B04125F167E4098
:10008E007FC27C017D207B05125F167E407FBD7C8A
:10009E00017D287B05125F167E407FC77C017D3077
:1000AE007B05125F167E407FCC7C017D387B04126F
:1000BE005F167E407FD07C017D407B04125F167EF2
:1000CE00407FD47C027DA07B09125F167E407FDDCF
:1000DE007C027DC07B07125F167E407FE47C027D32
:1000EE00E07B05125F167E407FE97C037D007B0579
:1000FE00125F167E407FEE7C037D207B05125F161D
:10010E007E407FF37C037D407B05125F167E407F31
:10011E00F87C037D607B09125F167E417F017C03B4
:10012E007D807B09125F167E417F0A7C037DA07B5A
:10013E0009125F167E417F137C037DC07B11125F17
:10014E00167E417F247C037DE07B07125F167E4185
:10015E007F2B7C047D007B07125F167E417F327CF5
:10016E00047D207B07125F167E417F397C047D4023
:10017E007B07125F167E417F407C047D607B0512FB
:10018E005F167E417F457C047D807B05125F167E67
:10019E00417F4A7C047DA07B05125F167E417F4F16
:1001AE007C047DC07B05125F167E417F547C047DEE
:1001BE00E07B05125F167E417F597C057D007B0535
:1001CE00125F167E417F5E7C057D407B09125F16B5
:1001DE009000297417F07F0312645E900028741942
:1001EE00F090002074B1F09000217491F0900022F4
:1001FE007403F0900023747FF090002404F09000BC
:10020E00257403F0E4900026F0900027F090003063
:10021E00740912530E7415F0A37403F0A37415121F
:10022E00530E7409F0A37403F0E4FFEFFD3395E071
:10023E00FC74302DF582740012536074102DF5820B
:10024E0074003CF583EEF00FBF08E0E4FFEFFD33E2
:10025E0095E0FC74382DF582740012536074182DDD
:10026E00F58274003CF583EEF00FBF08E090052098
:10027E00E4F0A374B4F0900522E4F0A374B4F0900B
:10028E0005247401F0A374E0F0900526E4F0A37445
:10029E0078F09005287402F0A37458F090052AE4C3
:1002AE00F0A3743CF090052C7402F0A37458F07413
:1002BE000790052EF0A3F0900530F0A3F0900532D4
:1002CE00F0A3F0900534F0A3F0900536E4F0A3749B
:1002DE003CF0900538740AF09005397428F09005BA
:1002EE003A7405F090053B740AF090053CF09005C9
:1002FE003D7428F09000A47401F0900B607415F01A
:10030E00A37411F09000A57401F0900B807415F099
:10031E00A37410F09000A67401F0900BA07415F069
:10032E00A37421F09000A77401F0900BC07415F027
:10033E00A37420F09000A87401F0900BE07415F0F7
:10034E00A37431F09000A97401F0900C007415F0B4
:10035E00A37430F09000AA7401F0900C207415F084
:10036E00A37441F09000AB7401F0900C407415F042
:10037E00A37440F09000AC7401F0900C60745312B2
:10038E0052FC74361252FC7438F0A3E4F0A374538A
:10039E00F0A3E4F09000AD04F0900C807453125270
:1003AE00FC7434F0A37421F0A37453F0A3E4F09022
:1003BE0000AF04F0900CC01252FA7430F0740312B5
:1003CE005358E4F09000B004F0900CE01252FA741E
:1003DE0030F07404125358E4F09000B104F0900D14
:1003EE00001252F274321252FC7452F0A37420F0C6
:1003FE009000B27401F0900D201252F27432F0A3FC
:10040E0074021253597420F09000B37401F0900DE1
:10041E004074531252FC7433F0A3E4F09000B40411
:10042E00F0900D601253237430F074021253039047
:10043E0000B57401F0900D801253237430F07405E2
:10044E001253039000B67401F0900DA01253237452
:10045E0030F0A374061253049000B77401F0900D9F
:10046E00C01253231253377498F0A3744B125304D3
:10047E009000B87401F0900DE012532312533774AC
:10048E0093F0A374181253049000B97401F0900EF7
:10049E00001253237430F0A37413125304A3747018
:1004AE00F0A37402F09000BA14F0900E2012532CA8
:1004BE007412F0A374701252FC7461F0A314F090D5
:1004CE0000BB7401F0900E4012532C74111253485D
:1004DE009000BC04F07461900E6012532E741412CE
:1004EE0053489000D104F09011001253237492F0EF
:1004FE00A3744BF0A37490F0A37402F0A37490F065
:10050E00A37432F07499A3F0A3F0A374601252FC9A
:10051E0074911252FC7491F0A3E412530490000FE4
:10052E007401F0125E4C7F01126F737F4012001641
:10053E007D2F7F0712672E7D0C7F0312672E7D3273
:0C054E007F0612672E7D1E7F0512672EAF
:01055A00227E
:0A5F16008E5A8F5B8C5C8D5D8B5EF4
:105F2000E4F9C3E55E6480F8E96480985028E9FFED
:105F30003395E0FEE55B2FF582E55A3EF583E49369
:105F4000FFE9FD3395E0FCE55D2DF582E55C3CF570
:065F500083EFF00980CC94
:015F56002228
:1056DD00AF6AEF3395E0FEE56975F008A42428F56F
:1056ED0082E43400F583E5822FF582E5833EF58370
:1056FD00E0FFE56AFD3395E0FC22AB66AD65AF6476
:10570D00223EF583E0FD74B82FF582741D3EF583BE
:10571D00EDF0056AE56A22EF3395E0FEEF25E0FF37
:10572D00EE33FE22A2E0CE13CE13223CF583EFF032
:05573D00056AE56A2287
:045BFD008C5B8D5CD4
:105C0100EF6043D201D202D20CE4F55D855C82855E
:105C11005B83E0FEA3E04E6027AF5D125724E55C95
:105C21002FF582E55B3EF583E0FEA3E0FF124460C1
:105C3100922920290B055DC3E55D6480949040CCD9
:065C4100C201C202C20C08
:015C4700223A
:045C48008C608D617E
:105C4C00EF6043D201D202D20CE4F5628561828509
:105C5C006083E0FEA3E04E6027AF62125724E5613B
:105C6C002FF582E5603EF583E0FEA3E0FF12446071
:105C7C00922D202D0B0562C3E5626480949040CC7C
:065C8C00C201C202C20CBD
:015C920022EF
:04446000AD07AC06F2
:10446400C22E780CEF088003125731D8FB540FF595
:10447400637808AF05AE04EF088003125731D8FB08
:10448400540FF5647804AF05AE04EF0880031257A7
:1044940031D8FB540FF565ED540FF566E563607193
:1044A400B40108125707123C518066E563B4020850
:1044B400125707126BA08059E563B403081257071B
:1044C4001238AA804CE563B40408125707126B41F2
:1044D400803FE563B405081257071224FA8032E5D9
:1044E40063B406081257071212698025E563B407FE
:1044F400081257071251028018E563B408081257CE
:10450400071258B9800BE563B409061257071269FC
:0345140058A22E7C
:014517002281
:103C51008F678D688B69E567B40113900020E0FFE1
:103C610012596F900020EFF0FD7F20023D0EE567B5
:103C7100B40211900021123D14900021EFF0FD7F5C
:103C810021023D0EE567B40311900022123D14900C
:103C91000022EFF0FD7F22023D0EE567B404109093
:103CA1000023123D1E900023EFF0FD7F23805EE58F
:103CB10067B40516900024123D1E900024EFF0FD1C
:103CC1007F247E001263F302658BE567B4061090D2
:103CD1000025123D28900025EFF0FD7F25802EE57F
:103CE10067B40710900026123D28900026EFF0FDE2
:103CF1007F268019E567B40819900027E0FFAB69BA
:103D0100AD6812596F900027EFF0FD7F277E0012FA
:103D110063F322E0FFAB69AD6812596F22E0FFAB9C
:103D210069AD6812596F22E0FFAB69AD6812596F36
:013D3100226F
:10596F00D22FAC07BD01047E018033BD02047E023D
:10597F00802CBD03047E048025BD04047E08801E98
:10598F00BD05047E108017BD06047E208010BD0764
:10599F00047E408009BD08047E808002C22FBB01B7
:1059AF0005EE4204800BEB7006EEF452048002C247
:0759BF002F302F03AF04227B
:0159C60022BE
:026BA0008B6701
:106BA200C22FEF7016ED7013E5677003025CDEE52D
:0B6BB20067B401077880E6FF125B1853
:016BBD0022B5
:0638AA008F678D688B6939
:1038B000E5677007123990E4FD801AE567B40107E7
:1038C0001239907D01800EE567B4020CAD69AF68D6
:1038D000126F037D02024F71E567B40306124DD1EA
:1038E000C21E22E567B40415AD69AF681264C68FC5
:1038F00043754205E542700302398F80F7E567643E
:10390000067017E5687013F56A1256DD74102DF510
:10391000827400125738B408F022E5676407701704
:10392000E5687013F56A1256DD74182DF58274007F
:10393000125738B408F022E56764087027E568700C
:1039400023E569701FF56AAF6AEF3395E0FE7410E6
:103950002FF582740012570EB408EC754201E5424F
:10396000602D80FAE56764097025E5687021E569D6
:10397000701DF56AAF6AEF3395E0FE74182FF5827B
:0F398000740012570EB408EC754201E54270FC5A
:09398F0022AD69AF68126F03223A
:106B41008F67AE03AF05E567D394004012E5679404
:106B510007500CAD06126F03AD07AF6712678222B3
:1024FA008F678D688B69E5677018E5687014E56900
:10250A0070057F01126F1FE569640160030226A747
:10251A008043E567701CE568B40117E56970057FBB
:10252A0004126F1FE569640160030226A77F040293
:10253A0026A4E5677029E56864027023E5697005D9
:10254A007F05126F1FE569640160030226A79000E8
:10255A000FE0B403057F010226A47F050226A4E545
:10256A0067B4011BE5687017E56970057F02126F91
:10257A001FE569640160030226A77F020226A4E51B
:10258A0067B4011CE568B40117E56970057F081294
:10259A006F1FE569640160030226A77F080226A46B
:1025AA00E56764017029E56864027023E5697005CE
:1025BA007F0A126F1FE569640160030226A7900073
:1025CA000FE0B403057F020226A47F0A0226A4E5CF
:1025DA0067B4021BE5687017E56970057F40126FE2
:1025EA001FE569640160030226A77F400226A4E56D
:1025FA0067B4021CE568B40117E56970057F10121B
:10260A006F1FE569640160030226A77F100226A4F2
:10261A00E56764027024E5686402701EE569700566
:10262A007F50126F1FE5696401707290000FE0B469
:10263A0003047F4080647F508060E567B40317E538
:10264A00687013E56970057F80126F1FE569640180
:10265A00704B7F808044E567B40318E568B40113C2
:10266A00E56970057F20126F1FE5696401702E7F8E
:10267A00208027E56764037024E5686402701EE51C
:10268A006970057FA0126F1FE569B4011090000FF1
:0E269A00E0B403047F8080027FA012001622AD
:101269008F678D688B69E5677017AD69AF68126F15
:10127900038E348F35D3E5359400E534940050F569
:1012890022E567B4011BE568B40116E5697007C278
:10129900307F01122ECAE569640160030214D68009
:1012A90058E5676401702BE56864027025E569708B
:1012B90007C2307F02122ECAE56964016003021475
:1012C900D690000FE0640370030214D6D2307F0277
:1012D9008031E5676401702EE56864037028E5696B
:1012E9007007C2307F03122ECAE5696401600302E8
:1012F90014D690000FE0B40306D2307F018004D2E7
:10130900307F03022ECAE5676401702DE568640425
:101319007027E569700CC2307F01122ECA7F401216
:101329006F1FE569640160030214D6D2307F011290
:101339002ECA7F40120016807CE5676401703AE589
:101349006864057034E569700CC2307F02122ECAD8
:101359007F10126F1FE569640160030214D69000C3
:101369000FE0640370030214D6D2307F02122ECA32
:101379007F10120016D22F803EE5676401703BE5AD
:101389006864067035E569700CC2307F03122ECA95
:101399007F50126F1FE569640160030214D6D230D1
:1013A9007F03122ECA90000FE0B403047F4080022D
:1013B9007F50120016C22F0269EAE567640270299C
:1013C900E56864017023E56970057F100214BDE5C5
:1013D90069B401057F100214C7E56964026003025C
:1013E90014D6D22F7F010214D3E56764027029E570
:1013F9006864027023E56970057F200214BDE56900
:10140900B401057F200214C7E56964026003021470
:10141900D6D22F7F020214D3E56764027029E568EA
:1014290064037023E56970057F400214BDE569B462
:1014390001057F400214C7E569640260030214D6FE
:10144900D22F7F030214D3E56764027023E5686431
:1014590004701DE56970047F808059E569B4010451
:101469007F80805AE56964027063D22F7F04805AB5
:10147900E56764027023E5686405701DE569700419
:101489007F048030E569B401047F048031E5696433
:1014990002703AD22F7F058031E5676402702EE52C
:1014A90068640670287D017F07124EE9401FE569CF
:1014B90070057F08026F60E569B401057F08026F56
:0E14C90073E569B40207D22F7F061229922222
:065102008F678D688B69C8
:10510800E567703BE5687037E569700690000F0445
:105118008021E569B4010A90000F7402F0D22F8053
:1051280047E56964027041C21E7FFF126F1F90003D
:105138000F7403F0C2307F02122ECAD22F8029E5E5
:105148006764017023E568701F7D077F05124EE9CB
:105158005016E569700BC200C2307F03122ECA8058
:1051680007E569B40102D200302F0C90000FE0FD72
:075178007F0F7E001263F3BC
:01517F00220D
:1058B9008F678D688B69E567700C1258FD749F2F8F
:1058C900F58274008019E567B4010C1258FD749FC4
:1058D9002FF58274008016E567B402091259053E56
:1058E900F583E4F022E567B403091259053EF5830F
:1058F9007401F022AD69AF68126F0322AD69AF6818
:0B590900126F03746F2FF582740022F0
:026958008F6747
:10695A00AF057804EF08800123D8FD4BF568E56799
:10696A00B40908E568B49903025455AD68AF6712D3
:02697A0065BBFB
:01697C0022F8
:0D6F0300EF75F00AA47C002DFFEC35F0FEC8
:016F1000225E
:046782008F688D6926
:10678600C3E569648094E4501BE4F56AC3E5696473
:1067960080F8E56A648098500BC22FAF6812299280
:0467A600056A80E818
:0167AA0022CC
:0D6F1100C296007F051268C21264F8D29685
:016F1E002250
:106DA800126F11EF20E0F9C296007F061268C2C286
:066DB800B60000D2962295
:106DBE00126F11EF20E0F9C296007F041268C2C272
:066DCE00B60000D296227F
:046056008E608F6168
:10605A00AE04AF058E638F64C296007F031268C2D6
:10606A00E560FF1268C2AF611268C2E4F5621264A9
:10607A00F8E5642562F582E43563F583EFF005629D
:09608A00E562C3942040E7D296C0
:0160930022EA
:085C93008E658F668C678D6839
:105C9B00126F11EF20E0F985656A85666BC296007D
:105CAB007F021268C2E567FF1268C2AF681268C252
:105CBB00E4F569E56B2569F582E4356AF583E0FF68
:105CCB001268C20569E569C3942040E7C2B60000BB
:025CDB00D2965F
:015CDD0022A4
:0A5677008E5A8F5B8C5C8D5D8B5E9C
:10568100C2AF126DA8126F11EF20E0F9855C608541
:105691005D61C296007F021268C2E55AFF1268C2BC
:1056A100AF5B1268C2E4F55FAF5EEF3395E0FEC316
:1056B100E55F9FEE6480F87480985014E561255F82
:1056C100F582E43560F583E0FF1268C2055F80D89A
:0B56D100C2B60000D296126DBED2AF30
:0156DC0022AB
:1063F3008E718F728D73C2AF126DA8126F11EF2061
:10640300E0F9C296007F021268C2E571FF1268C20A
:10641300AF721268C2AF731268C2C2B60000D296DE
:06642300126DBED2AF2293
:10610E00C2AFE4F55BF55CF55DF55EF55FF55AAE95
:10611E005EAF5FAC5BAD5C1260567420255CF55CC7
:10612E00E4355BF55B7420255FF55FE4355EF55E67
:0B613E00055AE55AC3948940D6D2AF41
:016149002233
:105E4C00C2AF756200756300756400E4F560F561BE
:105E5C00F55F126DA8AE63AF64AC60AD61125C937C
:105E6C0074202561F561E43560F56074202564F5D6
:105E7C0064E43563F563055FE55FC3948940D31231
:045E8C006DBED2AF66
:015E900022EF
:1057A1000500050105030507050F051F051E051C5D
:1057B100051805100201040E040A03060101040B79
:1057C1000304040F020304010302040D0200020298
:1057D100030004090404030503070100030304078C
:1057E100030104060402040C051605150000061544
:0E57F100062A060C06380633061E0612061798
:104CB5002430F58274003EF583EDFF3395E0FEE583
:104CC500822FF582E5833EF583E0FFEDFB3395E02A
:104CD500FA22AF411268C2C293126F6AD293D2AF61
:104CE500223EF583E0FC74B82FF582741D3EF583F2
:104CF500ECF00D221528E528D394002225E024A107
:104D0500F582E43457F583E49322E4F57CD20EC2B0
:104D150027C21DC21A227FA0126F1FE4F542C21ED0
:104D250022126F6AD2B67801EF0822122C44D2CA39
:0F4D3500D20ED22722ECFF3395E0FEEF78032257
:10416700200E2F900540E004F577D36480948150AA
:1041770003024227D3E5776480948F400375770F56
:10418700900029E0FF122C4490002AE0F576124DAA
:104197000F22301A58302712124CF94003024227D7
:1041A700C2CAC227D21D85762822301D0A124CF9B1
:1041B700506EC227C21D22AF7A157AEF700BC21A52
:1041C700E57625E0F528D21D22E57B30E0058576EA
:1041D700288008E57675F003A4F528AF7B7801EF12
:1041E70008800103D8FDF57BD227D2CA22D57708EC
:1041F700C20EE4F542C21E22057C7440257CF5827E
:10420700E43405F583E0124D01540FF57A740193F8
:10421700F57B700AD21DE57625E025E0F528D21A50
:014227002274
:10518000200E12900029E0FF122C4490002AE0F536
:1051900078124D0F22301A5130270F124CF9505D02
:1051A000C2CAC227D21D85782822301D0A124CF9A6
:1051B000504BC227C21D22AF7A157AEF7007C21A70
:1051C000C20EF54222E57B30E0058578288008E5AF
:1051D0007875F003A4F528AF7B7801EF0880010310
:1051E000D8FDF57BD227D2CA22E543124D01FA74CD
:0D51F0000193FBEA540FF57AEBF57BD21A20
:0151FD00228F
:1064F800E4F575D297F574C2B6126F6AAF75780174
:10650800EF08800123D8FDF5753097034375011214
:106518006F6AD2B60574C3E5746480948840D8AFB6
:0165280075FD
:01652900224F
:096F6A00000000000000000022FC
:1066D700C2B7E4FEC2B6126F6AEF30E704D2B580E4
:1066E70002C2B5124D26800123D8FDFF126F6A0E34
:0B66F700BE08E1C2B6D2B7D2B6D2B5E1
:016702002274
:0D001600C2AFEF4227AF271266D7D2AF224C
:0E6F1F00C2AFEFF45227AF271266D7D2AF22CF
:1068C200E4FEC2B6126F6AEF30E704D2B58002C2AC
:1068D200B5124D26800123D8FDFF126F6A0EBE0845
:0568E200E1D2B6D2B5C1
:0168E700228E
:096F7300C2AFEF4241124CD722DB
:0A6F6000C2AFEFF45241124CD722E9
:102C4400EF123A5E2CAC012CB3022CBA032CC10453
:102C54002CC8052CCF062CD6072CDD082CE4092C17
:102C6400EB0A2CF20B2CF90C2D000D2D070E2D0E5A
:102C74000F2D15102D1C112D23122D2A132D311457
:102C84002D38152D3F162D46172D4D182D54192D61
:102C94005B1A2D621B2D691C2D6B1D2D721E2D7947
:102CA4001F2D802000002D6975CB8E75CAC6227534
:102CB400CB9575CA772275CB9B75CA692275CBA053
:102CC40075CABA2275CBA675CA332275CBAB75CA41
:102CD400632275CBB075CA022275CBB475CAA32220
:102CE40075CBB875CAFA2275CBBC75CAD82275CB18
:102CF400C075CAA82275CBC475CA362275CBC775F0
:102D0400CA862275CBCA75CABC2275CBCD75CAB426
:102D14002275CBD075CA762275CBD375CA3022758D
:102D2400CBD575CAB22275CBD875CA132275CBDA46
:102D340075CA522275CBDC75CA7D2275CBDD75CA86
:102D44006E2275CBE075CA542275CBE275CA1B227C
:102D540075CBE375CAC32275CBE575CA5E2275CB04
:102D6400E675CADA22801C75CBE875CA902275CB49
:102D7400EA75CAD92275CBEC75CA092275CBED75F3
:0A2D8400CA292275CBE875CA412266
:10002600C3EF648094A15008EF25E025E0F528226F
:04003600E4F52822A3
:0237B3008F5A2B
:1037B500900118E0FFE55A7006E545D39F5012E5E4
:1037C5005A640160030238A9E546D39F50030238C5
:1037D500A9E55A7018C3E5459FF55D74602FF5821C
:1037E500E4341EAD82F55E8D5F7F40801BE55AB4E3
:1037F5000119C3E5469FF55D74B02FF582E4341ECB
:10380500AF82F55E8F5F7F101200167FF47E011286
:103815006CC47D207F0512672E7D1A7F0812672EE6
:103825007FC87E00126CC4E4F55BE55BC3955D5013
:1038350061055FE55FAE5E7002055E14F5828E83FD
:10384500E0F55C123A5E38860038640A38680B3851
:103855006E0C38740D387A0E38800F0000388CE401
:10386500FD80277D5F7F0780227D5E7F06801C7D32
:103875000A7F0280167D327F0280107D467F02809E
:103885000A7D0A7F038004AD5CE4FF12672E055BA9
:103895008098E55A70047F408007E55AB401057F9A
:0438A50010126F1F6F
:0138A90022FC
:10507F00200E10754406901DB8E06003D20E22E496
:10508F00F54222E528D394004003152822C2CA1501
:10509F0044E54414603D14603214601D146015140F
:1050AF007049901DB8E0FF7003F54222122C449016
:1050BF001DB9802F901DBA8015901DBBE0FF7003A6
:1050CF00F54222122C44901DBC8018901DBDE0FFAC
:1050DF00020026901DBEE0FF7003F54222122C4401
:1050EF00901DBFE0FF120026D2CA22E4F542C2CAC9
:0350FF00C20E22BC
:1066A900900028E0FF6026200E07124D307528144F
:1066B90022E528D394004003152822202708D2CAAE
:0E66C900752814D22722C2CA75287DC2272246
:10664B00200E0C7F1C124D3075286475793C22E5A9
:10665B0028D394004003152822AF791579D3EF6422
:0E666B00809480400475286422C20EE4F5423B
:0166790022FE
:10635000E54214601C14601C14601F146022146059
:106360002224057021C2CAC20EC227C21DE4F54410
:106370002202507F1266A9D21E22124167D21E222B
:0763800002664B125180225E
:10645E00BF010790002A7418F022BF020790002A8D
:10646E007412F022BF030590002A8014BF04079017
:10647E00002A740BF02290002ABF05047409F02242
:04648E00740CF02278
:024FF900AC0703
:104FFB00C3EC64809480404AEC64809488504320D6
:10500B002B21E4FD124D3AC333CE33CED8F9124CDB
:10501B00B574102BF58274003AF583EFF00DBD08D3
:10502B00E3801FE4FD124D3AC333CE33CED8F912D1
:10503B004CB574182BF58274003AF583EFF00DBD67
:10504B0008E3202B16E4FDEDFF3395E0FE74102FE3
:10505B00F5827400124CE6BD08ED22302B15E4FDF1
:10506B00EDFF3395E0FE74182FF5827400124CE6B9
:03507B00BD08ED80
:01507E00220F
:105455007D3F7F0912672E7D507F0812672E906F62
:105465009C1254BC7D5B7F0612672E906F9D125473
:10547500BC906F9EE493FDE4FF12672E906F9FE44E
:105485009324BE601414601514601814601B146016
:105495001E240570217D0A80067D3280027D467FAF
:1054A5000280107D0A7F03800A7D287F0380047DAA
:1054B500467F0312672E22E493FDE4FF12672E2236
:105F98008F5BE55B7005D22DFF8009E55BB40107D7
:105FA800D22D7F01125A757D4B7F0212672E7D021A
:105FB800E4FF12672E7D32E4FF12672E125455E576
:105FC8005B70028005E55BB401057F40126F1F22FC
:103D3200A209300501B350307D017F04124EE950D3
:103D42002320050E30090B9000A4E0FF7C0B7D6060
:103D5200800F30050F20090C9000A5E0FF7C0B7D41
:103D620080125C48A2099205A20A300601B35030C3
:103D72007D027F04124EE9502320060E300A0B907A
:103D820000A6E0FF7C0B7DA0800F30060F200A0CFE
:103D92009000A7E0FF7C0B7DC0125C48A20A92064D
:103DA200A20B300701B350307D037F04124EE9505D
:103DB2002320070E300B0B9000A8E0FF7C0B7DE068
:103DC200800F30070F200B0C9000A9E0FF7C0C7DC8
:103DD20000125C48A20B9207A20D300801B35030CA
:103DE2007D047F04124EE9502320080E300D0B9003
:103DF20000AAE0FF7C0C7D20800F30080F200D0C04
:103E02009000ABE0FF7C0C7D40125C48A20D920852
:013E1200228D
:10658B00534103900024E0FE543FFF780408800140
:10659B0023D8FD54F0FFEE30E403430704900024AE
:0F65AB00E030E503430708EF4241C2AF124CD77F
:0165BA0022BE
:022992008F6B49
:10299400302F05756CF48003756C64E56B6401700D
:1029A40029AF417803EF08800123D8FD3392307FAB
:1029B4001020300B122AAE7F10126F60022AA6126A
:1029C4002AB97F10126F73022AA6E56B640270287D
:1029D400AF417802EF08800123D8FD3392307F2085
:1029E40020300A122AAE7F20126F608008122AB9A2
:1029F4007F20126F73022AA6E56B64037028AF412F
:102A04007801EF08800123D8FD3392307F402030D5
:102A14000A122AC47F40126F608008122ACF7F40B6
:102A2400126F73022AA6E56B6404701EE5413392AB
:102A3400307F8020300A122AC47F80126F608008A1
:102A4400122ACF7F80126F738058E56B640570275C
:102A5400AF417805EF08800123D8FD3392307F041D
:102A640020300A122ADA7F04126F608008122AE5E5
:102A74007F04126F73802BE56B6406702CAF417872
:102A840004EF08800123D8FD3392307F0820300AF8
:102A9400122ADA7F08126F608008122AE57F081272
:092AA4006F73AF6C7E00126CC46C
:102AAD0022126F73AF6C7E00126CC422126F60AF76
:102ABD006C7E00126CC422126F73AF6C7E00126CB0
:102ACD00C422126F60AF6C7E00126CC422126F7341
:102ADD00AF6C7E00126CC422126F60AF6C7E001260
:032AED006CC42294
:105DBB00900024E030E0057F10126F73900024E018
:105DCB0030E1057F20126F73900024E030E2057FF5
:105DDB0040126F73900024E030E3057F80126F73E5
:105DEB00900024E030E4057F04126F73900024E0F0
:095DFB0030E5057F08126F7322E8
:106D150030030A124D1BC203C211C21E22300409E0
:0A6D2500124D1BC204C213C21E224D
:1065BB008F708D71E570B4011FE5717003125CDE95
:1065CB00E571B401077880E6FF125B18E571B43210
:1065DB000E7FF47E01026CC4AD71AF7012672E2278
:10672E00EFFEEDFF1280008E2D8F2E1253E075744A
:10673E0032AF741574EFD39400400EE4F573E57325
:09674E00C3943A50EC057380F588
:01675700221F
:1053E000D2A8AFA875A881C214852E82852D83E42A
:1053F00093C4540FFE4306F08E80C284D28500C24F
:10540000870000D287007580FF7580FEC284C28548
:1054100000C2870000D287007580FFD2147D407CD7
:105420001FE4FE30B40D0EBE32F9ED1D70011CED0F
:105430004C70EE7C1F7D40E4FE20B40D0EBE32F9B0
:10544000ED1D70011CED4C70EE8FA8C2A87F0A7E86
:0454500000126CC416
:015454002235
:106758007580FDC284C28500C28700000000D28710
:10676800007580FF7F0A7E00126CC47F997E091233
:0A67780080008E2D8F2E1253E022B8
:10422800D284D285C286A2809217A2819220A282CD
:104238009218A2839221D2862001537D027F011217
:104248004EE940137D037F01124EE9400A301707FB
:10425800301932D22480377D027F01124EE9500F87
:1042680030170C302009301904D224802180167DA3
:10427800037F01124EE9501220170330200C301929
:1042880004D22480091267FC8004C219C2242002C7
:104298004E7D027F02124EE940127D037F02124ECC
:1042A800E94009301806301B2FD225227D027F02F3
:1042B800124EE9500E30180B302108301B03D2255E
:1042C8002280157D037F02124EE9500F201803301B
:1042D8002109301B03D22522026824C21BC22522D1
:1067FC00753D1E753E60E4FFE53E2FF582E4353DA8
:10680C00F583E4F00FBF50F0753D1E753E60E4F566
:07681C0045C226C211D2198A
:016823002252
:10682400753F1E7540B0E4FFE5402FF582E4353F27
:10683400F583E4F00FBF10F0753F1E7540B0E4F52A
:0768440046C228C213D21B5B
:01684B00222A
:106C5200C284D285C286A2809209A281920AA282AD
:0D6C6200920BA283920DD286D284D285229D
:10618600E57E2560F582E4357DF5832274FF123ABB
:1061960034E4FBFAF9F8C3023A21057F7480257EC0
:1061A600F57EE4357DF57D22F582E4341DF5832206
:0B61B600757F01757D00757E20E422DE
:1042E8007D027F07124EE950057F04126F60C229D4
:1042F800D223E4F5427FE87E03126CC4C298C2AFB1
:10430800C2307F03122ECA755E7F755D96755C9804
:10431800755B00785B126192504430983E1200063B
:10432800126E76EF14601824F0602624C1600B2406
:10433800F670287F06126F858021126270801C7FBC
:1043480006126F85126A3012658B125E4CD2298074
:104358000A7F06126F85125AC8D2293029B5E47827
:1043680085F6D2307F01122ECA7F40120016C22F66
:104378001269EA7D467F0212672E7D1E7F0712674B
:104388002E7D147F0812672E7D327F0312672EC29E
:0D439800307F03122ECA7FFF126F1FC22359
:0143A50022F5
:105AC8001261B6F55F7F02126F85E57F2402F561EA
:105AD800AF7F126F85E4F560126186E0FF126F8573
:105AE800126186E02561F5610560E560C394804038
:105AF800E7AF61126F857F03126F85126F8DEF64B8
:0F5B080015600C1261A0055FE55FC3942240B6E3
:015B1700226B
:106A30001261B6F55F12649250077F06126F85806F
:106A4000057F15026F851261A0055FE55FC3942283
:026A500040E321
:016A52002221
:10649200E4F560126F8D74D025601261AEEFF005E5
:1064A20060E560C3948440EB126E54901E52E0B5D6
:1064B2000710AE7DAF7EBE0504BF200100126CA89E
:0364C200D322C31F
:0164C50022B4
:106CA800E4FF74D22FF582E4341DF583E0FEE57E1F
:0B6CB8002F12618AEEF0000FBF80E792
:016CC30022AE
:106E5400E4FFFE74D02E1261AEE02FFF0EBE82F36B
:016E6400220B
:10627000E4F55FF5657564E0756393756204F56137
:10628000786112619250213098F61200068F60E515
:106290006064046013AF65056574D02F1261AEE5CC
:0862A00060F0255FF55F80D876
:0162A80022D3
:04000600AF99C29854
:01000A0022D3
:086F85003099FDC2998F992299
:076F8D003098FDAF99C29896
:016F940022DA
:106D62000C0102030405060708090A0B0C010203C1
:086D72000405060708090A0BDD
:1067AB00AF5FEF3395E0FE75F007EF123A52EE75DF
:1067BB00F007A42583F583E0227883E6FF126D4969
:0967CB00EF22C295D297D2AF2251
:1068E800C22CC2AF126F957F83126D7A126B611240
:1068F80067CD7884E66F600B125ED4302B05125F8B
:05690800D8922CA22C26
:01690D002267
:105FD8007984E778876660367884E6FF7887F6EF15
:105FE8007013E552C3940A500C7D077F04124EE9E2
:105FF8005003125E917D057F04124EE95010E54171
:1060080054036005123FCAD322123FCAC322C322D7
:103FCA00E4F55F900A501267AB700302408E900AC4
:103FDA00511267B26016788166600302408E900AB9
:103FEA00521267AB788866600302408EAF5FEF3388
:103FFA0095E0FE900A531267B2FF7880E6FEEF6EF4
:10400A006020EF601DB4080BEED394014005EE94D6
:10401A0007400FEF6409706CEE64016005EE6407F7
:10402A007062AF5FEF3395E0FE900A541267B2FFF9
:10403A00F46006EF788366704BE55FFD3395E0FC2C
:10404A00900A5575F007ED123A52EC1267BA788465
:10405A00667031D201D20274BD2DF58274003CF52E
:10406A0083E0FFC007EDAE047805C333CE33CED864
:10407A00F92480F582740E3EAD82FCD007125C48AA
:10408A00C201C202055FC3E55F64809493500302D4
:02409A003FCD18
:01409C002201
:105E91007D087F04124EE9500D7883E6FF126D49AB
:105EA100EFC39407402CD2307F01122ECA7F4012DB
:105EB1000016C22F1269EAD201D202E4FD7F0A1252
:105EC1004F71C201C2027F50126F1FC2307F011297
:035ED1002ECA22B4
:105ED400C2AF126F957FBF126D7A126B617884A680
:105EE40007126B617884A607126B617883A6071288
:105EF4006B617888A607126B617881A607126B61C3
:105F04007880A607126B617882A607126F951267D4
:025F1400CD229C
:10591400C2AF126F957F8E1259637F90126D7A7F9A
:10592400A7126D7A126F957FBE126D7AE4FF126D25
:105934007A7884E6FF126D7A7883E6FF126D7A78BE
:1059440088E6FF126D7A7881E6FF126D7A7880E638
:10595400FF126D7A7882E6FF1259631267CD221224
:0B5964006D7AE4FF126D7A126F95223D
:105B18008F72E572B401047D63803EE572B40206BB
:105B28007D087F068035E572B403067D317F0880E5
:105B38002AE572B404067D617F08801FE572B4050A
:105B4800067D257F088014E572B406067D597F031B
:0F5B58008009E572B407077D487F0712672E2288
:026D4900AE0793
:106D4B00EE54F0FF780408800103D8FD75F00AA417
:066D5B00FFEE540F2FFFB4
:016D6100220F
:105CDE001267C4906D6293FF1235B878841267C64E
:105CEE00601B78841267C6C3940A50077D327F0604
:105CFE0012672E7884E6FF126D491235B81267C40A
:105D0E00C3940C50067D0A7F0280047D507F0612DC
:0A5D1E00672E7D507F0512672E22CC
:105A1F007FF47E01126CC47D097F0612672E788198
:105A2F00125A657D0E7F0312672E7D357F06126732
:105A3F002E7D097F0612672E7888125A657D1E7F8C
:105A4F000912672E7D1E7F0712672E7882E6FF12DE
:105A5F006D491235B822E6FF126D491235B87FF441
:065A6F007E01126CC4224E
:076F9500C2B6C295D295229D
:106D7A00E4FEC297EF30E002D297C2B6D2B6EFC3B2
:066D8A0013FF0EBE08EC31
:016D900022E0
:106B6100E4FFD297FED2B6C2B6A297E433C4333360
:0F6B7100335480FDEFC313FFED42070EBE08E65D
:016B800022F2
:10585C00EF3395E0FE74702FF58274003EF583E013
:10586C00FF22AF5AEF3395E0FEEF222460F58274ED
:10587C00013EAD82FCD22922900520E0F547A3E041
:10588C00F548222450F58274053EAD82FC2290002E
:10589C00BAE0FF7C0E7D2022D222D201E4FF22C28C
:0D58AC0001C2227F1922D222D2307F0222B7
:10283100E5527008126F498F5202292CE552B405F6
:10284100081245188F5202292CE552B40B08126C5C
:10285100DF8F5202292CE552B40A08125D288F52EB
:1028610002292CE552B40F081260D18F5202292C93
:10287100E552B414081223408F5202292CE552B4B8
:102881001908126BBE8F5202292CE552B41E081290
:102891006A998F5202292CE552B42308126AFF8FDC
:1028A1005202292CE552B42807126F2D8F52807BDA
:1028B100E552B42D071268748F52806FE552B4321D
:1028C100071262A98F528063E552B43E07126BDC96
:1028D1008F528057E552B43C07126E1E8F52804BC7
:1028E100E552B43307126ADD8F52803FE552B4419D
:1028F10007126EA78F528033E552B44C07126EB7A0
:102901008F528027E552B44407126EC78F52801B45
:10291100E552B437071257428F52800FE552B4394E
:10292100071254C58F528003E4F552E55370061225
:10293100000E8F5322E553B40506126F7C8F53228C
:10294100E553B40A06126ED78F5322E553B40F062E
:10295100126EE68F5322E553B41406123B6E8F5369
:1029610022E553B43D06126BFA8F5322E553B43F6F
:10297100061265EB8F5322E553B4430612684C8F60
:102981005322E553B44D06126B208F5322E4F553C5
:012991002223
:0D6F490090052AE0F52BA3E0F52C7F052232
:10451800302414201011C21C7D047F01124EE95072
:10452800037F0B227F0A227F0812638750061245F9
:10453800CE7F0022202408301005C2107F05227D7E
:10454800057F06124EE9501EE5394538701890006F
:10455800B5E0FF7C0D7D80125C4890052EE0F538B3
:10456800A3E0F53980517D067F06124EE9501EE51D
:104578003C453B70189000B6E0FF7C0D7DA0125CB6
:1045880048900530E0F53BA3E0F53C802A7D077FA5
:1045980005124EE9500B300008E52C452B7002C27D
:1045A80000300F08E52C452B7002C20F7885E6B461
:1045B80005057F041251FEE551700875510AD22B8A
:0645C8001268E87F0522E5
:106CDF00200F1590053BE0F54E2024037F0522E59C
:0B6CEF004ED3940050F3D20F7F0A2216
:105D28007D077F05124EE9500C7D077F05124EE96D
:105D3800503230002F7D017F01124EE95026D230BB
:105D48007F01122ECA7F011200167D027F07124EB4
:105D5800E950057F04126F739000A0E0FF7C0A7D74
:0A5D6800E0125C481258847F0F22FD
:1060D100302437E5484547700C7D087F01124EE9B1
:1060E10050037F372230030EE53A700A126D157F97
:1060F1000112001680113026037F14227885E6B440
:0D61010005057F031251FE7F0F227F14223F
:1023400090053DE0F54B7F01126F1F126D157D0268
:102350007F07124EE95009E54B70057F04126F604C
:102360009000A1E0FF7C0B7D00125C48D22B12682C
:10237000E8E545700302246A7C017D001224F250D6
:10238000037F3E227C017D501224D250037F3C22E9
:102390007C017D581224D250037F3C227C017D10A9
:1023A0001224DA50081224E250037F33227C017D8C
:1023B000201224DA500B9000BBE0FF7C0E7D4080A1
:1023C000207C017D281224EA500512589A80127C44
:1023D000017D301224EA50129000B9E0FF7C0E7D9E
:1023E00000125C481267FC7F00227C017D40D229EC
:1023F000E4FF1247E3500C7D067F04124EE95003C0
:102400007F4C227C017D381224F250037F44227CD1
:10241000017D18C229E4FF1247E3500C7D057F01BE
:10242000124EE950037F4122E4F55A12586E7803A8
:10243000C333CE33CED8F9125877E4FF1247E350B6
:102440001BAF5A12585CC00712586E7805C333CEC2
:1024500033CED8F912588FD007125BFD055AC3E569
:102460005A648094A840C47F19221224E2500C7D43
:10247000077F05124EE9504B3000487885E670041E
:102480007F0180087885E6B404077F021251FE8040
:102490002F7885E6B40704760180257D037F061238
:1024A0004EE9501CE557455670169000AFE0FF7C92
:1024B0000C7DC0125C48900532E0F556A3E0F5575C
:1024C0007F19227D077F05124EE950052000027F0B
:0124D0000506
:1024D10022D229E4FF1247E322D229E4FF1247E383
:1024E100227D077F05124EE922D229E4FF1247E33C
:0924F10022C229E4FF1247E32294
:106BBE003026031267FC7D077F05124EE950062032
:0E6BCE0000037F0522900538E0F54E7F1E2261
:106A9900E54E70037F23227D027F07124EE95009DC
:106AA900E54B70057F04126F603024037F0A227F53
:026AB9001E229B
:106AFF001258847D067F01124EE9500C9000ACE0D5
:106B0F00FF7C0C7D60125C48900539E0F54E7F2DBF
:016B1F002253
:0E6F2D007FA0126F1F900539E0F54E7F2D22D8
:10687400D22B1268E87D027F07124EE95009E54BDE
:1068840070057F04126F60E54E70037F322230245E
:07689400037F0A227F2D2281
:1062A900301E037F32227D047F06124EE9501FE51E
:1062B90055455470199000B0E0FF7C0C7DE0125CEC
:1062C90048900534E0F554A3E0F5557F3222C230F9
:0862D9007F01122ECA7F002292
:106E1E0020220CD222E4FF12055BC2227F00227FC9
:026E2E003C2204
:106BDC00202218D2227F40120016D201121D87C229
:0E6BEC00017F40126F1FC2227F19227F3E22BE
:106EA70020220A1258A41237B31258AB227F41226C
:106EB70020220A1258A412614A1258AB227F442298
:106EC70020220A1258A412560E1258AB227F4422CF
:05000E0000007F052247
:096F7C003025037F0A227F052263
:0F6ED7009000A2E0FF7C0B7D20125C487F0F2211
:0F6EE6003025093028037F14227F0F227F1422CA
:103B6E009000A3E0FF7C0B7D40125C48E54670039D
:103B7E00023C467D017F03124EE950707C017D08A8
:103B8E00C2297F011247E350037F3F227C017D5003
:103B9E00123C4950037F3D227C017D58123C495016
:103BAE00037F3D227C017D40D2297F011247E350E5
:103BBE000C7D067F04124EE950037F4D227C017D61
:103BCE0028D2297F011247E3500912589A125C48F5
:103BDE007F00227C017D18C2297F011247E3500C21
:103BEE007D057F02124EE950037F43227D027F0343
:103BFE00124EE95043E4F55AAF5A1258707803C387
:103C0E0033CE33CED8F91258777F011247E3501DC9
:103C1E00AF5A12585CC007AF5A1258707805C333AA
:103C2E00CE33CED8F912588FD007125BFD055AC38A
:0A3C3E00E55A648094A840C07F009E
:093C480022D2297F011247E32278
:106BFA00202218D222C2307F01122ECA7F01126FC0
:0E6C0A001F7F0112055BC2227F00227F3D2208
:1065EB0020222A1258B2122ECA7FF47E01126CC4DA
:1065FB007F10120016D202121B86C2027F10126F7E
:10660B001FC2307F02122ECAC2227F00227F3F227E
:10684C002022221258B2122ECA7FF47E01126CC47E
:10685C00D2027F011237B3C202C2307F02122ECA9B
:08686C00C2227F00227F4322BB
:106B200020221B1258B2122ECAD2027F0112614AD1
:106B3000C202C2307F02122ECAC2227F00227F4DC3
:016B40002232
:10553500AF5AEF3395E0FE22900520E0F547A3E052
:10554500F54822900522E0F549A3E0F54A222460BA
:10555500F58274013EAD82FCD2292274702FF5824A
:1055650074003EF583E0FF22C202C2227F19222485
:1055750050F58274053EAD82FC22900536E0F53289
:10558500A3E0F53322055AC3E55A648094A822D2D4
:0D55950022C2307F0122D222C2307F0222CA
:10326500E5527006126ABB8F5222E552B40506126A
:1032750036B78F5222E552B40B0612689B8F522245
:10328500E552B40A061243A68F5222E552B40F0640
:10329500126E308F5222E552B411061259C78F5261
:1032A50022E552B412061252788F5222E552B41416
:1032B50006120A548F5222E552B4190612667A8F05
:1032C5005222E552B41E0612661B8F5222E552B4F5
:1032D5002306125F578F5222E552B42806126F3B20
:1032E5008F5222E552B42D061261C18F5222E5524A
:1032F500B432061262E18F5222E552B43C06126ED8
:10330500428F5222E552B43D06126CFA8F5222E5E5
:1033150052B43E0612697D8F5222E552B43F061221
:103325006E658F5222E552B44106126B818F52228F
:10333500E552B44306126A538F5222E552B44C0645
:10334500126D2F8F5222E552B44D06126A768F52B6
:1033550022E552B437061257428F5222E552B4394C
:10336500061254C58F5222E552B438061267038FF0
:103375005222E552B43306126ADD8F5222E552B469
:0C3385004406126D918F5222E4F5522292
:106ABB0090052AE0F52BA3E0F52C7D067F02124E04
:106ACB00E9500C90052CE0F529A3E0F52AD21F7FA5
:026ADB00052292
:1036B700302414201011C21C7D047F01124EE950E2
:1036C700037F0B227F0A22302514201211D21C7D82
:1036D700047F02124EE950037F0B227F0A227F08E4
:1036E70012638750061245CE7F002220240830102F
:1036F70005C2107F0522202508301205C2127F055A
:10370700227D057F06124EE9501EE53945387018AF
:103717009000B5E0FF7C0D7D80125C4890052EE09F
:10372700F538A3E0F53980757D067F06124EE9501E
:103737001EE53C453B70189000B6E0FF7C0D7DA070
:10374700125C48900530E0F53BA3E0F53C804E7DE8
:10375700077F05124EE9500D30000AE52C452B7006
:1037670004C200800B300F08E52C452B7002C20FF6
:103777007D067F02124EE95019301F16E52A4529AA
:103787007010C21F9000BCE0FF7C0E7D60125C4889
:10379700800B7885E6B405057F041251FEE551706C
:0C37A7000875510AD22B1268E87F052239
:10689B00200F2190053BE0F54E202406201C037FA2
:1068AB000522202506301C037F0522E54ED39400DC
:0768BB0050E7D20F7F0A2213
:1043A6007D077F05124EE950127D077F05124EE903
:1043B6004003024457200003024457201C3FD230DA
:1043C6007F03122ECA7F0F126F1F90000FE0B402F8
:1043D600047F05800990000FE0B403057F011200F9
:1043E6001612553D7D027F07124EE950057F0412D5
:1043F6006F739000A0E0FF7C0A7DE0804E301C5178
:1044060090000FE0FF64026005EF640370437F0FC6
:10441600126F1F7F05126387400BD2307F01122E69
:10442600CA7F028009D2307F03122ECA7F0A120089
:10443600167D027F07124EE950057F04126F731234
:1044460055489000A2E0FF7C0B7D20125C487F0F50
:0A4456002212553D1255487F0F2237
:106E3000201C063024037F1122301C053025027FE0
:026E400012221C
:1059C700302452E5484547700C7D087F01124EE9A7
:1059D70050037F3722300329E53A70257FA0126FE5
:1059E7001F90000FE0B401047F01800990000FE0D1
:1059F700B402057F05120016E4F542C21EC20380F9
:105A0700113026037F14227885E6B405057F03123B
:085A170051FE7F11227F1422D1
:10527800301C1030240D20100A7F0A126F1FC21C28
:105288007F0A22301C4C3025492012463003031275
:105298006D15E54A4549700C7D087F02124EE950AC
:1052A800037F3822300417E53A70137FA0126F1F6E
:1052B8007F02120016E4F542C21EC2048011302893
:1052C800037F14227885E6B405057F031251FE7F1B
:1052D8001222201C1230250F20120CD21CC2307F43
:0A52E80002122ECA7F0A227F142250
:100A540090053DE0F54B7F0F126F1F201C0C90009A
:100A6400A1E0FF7C0B7D00125C48301C0C9000A3BD
:100A7400E0FF7C0B7D40125C48E542B403037F1425
:100A840022126D15E4F5427D027F07124EE95009EA
:100A9400E54B70057F04126F60D22B1268E8301C9E
:100AA40003020B97E5457003020B977C017D00124E
:100AB4000D1E50037F3E227C017D50120CEE50032C
:100AC4007F3C227C017D58120CEE50037F3C227C3B
:100AD400017D10120CF65008120D0650037F3322CC
:100AE4007C017D20120CF65003020BFE7C017D2854
:100AF400120D0E500C9000BAE0FF7C0E7D20020C0B
:100B0400077C017D30120D0E500C9000B9E0FF7C83
:100B14000E7D00020C077C017D40D229E4FF1247C0
:100B2400E3500C7D067F04124EE950037F4C227C77
:100B3400017D38120D1E50037F44227C017D18C2B2
:100B440029E4FF1247E3500C7D057F01124EE95062
:100B5400037F4122E4F55A125535EF7803C333CEAF
:100B640033CED8F9125553E4FF1247E3501D125502
:100B740035125560C007125535EF7805C333CE33AF
:100B8400CED8F9125574D007125BFD12558A40C7AE
:100B94007F1922201C03020C8AE5467003020C8A8A
:100BA4007D017F03124EE94003020C427C017D0863
:100BB400C2297F011247E3500F7F50120016D23032
:100BC4007F02122ECA7F3F227C017D50120CFE5000
:100BD400037F3D227C017D58120CFE50037F3D2291
:100BE4007C017D10120D165008120D0650037F3340
:100BF400227C017D20120D1650129000BBE0FF7C78
:100C04000E7D40125C481267FC7F00227C017D400F
:100C1400D2297F011247E3500C7D067F04124EE96E
:100C240050037F4D227C017D18C2297F011247E3C6
:100C3400500C7D057F02124EE950037F43227D0252
:100C44007F03124EE9503CE4F55A125535EF780310
:100C5400C333CE33CED8F91255537F011247E35034
:100C64001D125535125560C007125535EF7805C36E
:100C740033CE33CED8F9125574D007125BFD12551A
:100C84008A40C77F1922120D265008120D26504B98
:100C94003000487885E670047F0180087885E6B4E2
:100CA40004077F021251FE802F7885E6B40704768C
:100CB4000180257D037F06124EE9501CE5574556F9
:100CC40070169000AFE0FF7C0C7DC0125C4890056C
:100CD40032E0F556A3E0F5577F19227D077F051210
:090CE4004EE950052000027F05D5
:100CED0022D229E4FF1247E322D229E4FF1247E37F
:100CFD0022D2297F011247E3227D077F05124EE99B
:100D0D0022D229E4FF1247E322D2297F011247E3C1
:100D1D0022C229E4FF1247E3227D077F05124EE927
:010D2D0022A3
:10667A00C219C2307F02122ECA3026051267FC8068
:10668A00063028031268247D077F05124EE950065A
:0F669A002000037F0522900538E0F54E7F1E2279
:10661B00E54E70037F23227D027F07124EE950095E
:10662B00E54B70057F04126F603024062010037F4A
:10663B000A22302508201205D21C7F0A227F1E2237
:105F5700201C0512553D80031255487D067F01120E
:105F67004EE95024E5427020201C0B9000ACE0FF66
:105F77007C0C7D60800C301C0C9000ADE0FF7C0C2D
:105F87007D80125C487F2822900539E0F54E7F2DF1
:015F970022E7
:0E6F3B007FA0126F1F900539E0F54E7F2D22CA
:1061C100D22B1268E87D027F07124EE95009E54B98
:1061D10070057F04126F60E54E601D3024062010AB
:1061E100037F0A2290000FE0640160093025062038
:0B61F10012037F05227F2D227F322247
:1062E100301E037F32227D047F06124EE9501FE5E6
:1062F10055455470199000B0E0FF7C0C7DE0125CB4
:1063010048900534E0F554A3E0F5557F3222C230C0
:086311007F01122ECA7F002259
:106E420020220CD222E4FF12055BC2227F00227FA5
:026E52003C22E0
:10697D0020221FC2307F02122ECAD2227F40120067
:10698D0016D201121D87C2017F40126F1FC2227FD6
:05699D0019227F3E22DB
:106E650020220BD222D202121B8612556D227F3FA1
:016E750022FA
:106CFA00202215125594122ECA7F40126F1F7F014F
:0B6D0A0012055BC2227F00227F3D22A9
:106B810020221912559B122ECA7F10126F1FD2019B
:0F6B9100E4FF1237B3C201C2227F19227F4122D3
:106A530020221D125594122ECA7F40126F1FD2306E
:106A63007F02122ECAD2027F011237B312556D2252
:036A73007F43223C
:106D2F0020221412559B122ECAD201E4FF12614A7F
:0A6D3F00C201C2227F19227F412207
:106A760020221D125594122ECA7F40126F1FD2304B
:106A86007F02122ECAD2027F0112614A12556D226E
:036A96007F432219
:106D910020221112559B122ECAD202E4FF12560E66
:076DA10012556D227F442210
:10574200D2107D027F07124EE950057F04126F606E
:1057520090000FE0FF64016004EFB4030E7F0112BA
:105762006F1F7F401257917F01801390000FE0B4AA
:10577200020F7F05126F1F7F501257917F03126F26
:10578200607F50126F1F30150312557F7F3922122E
:0F5792000016C22F1269EAE4FD7F07124F712241
:1054C50030241130150BE53345327005C2311269B0
:1054D500A27F3922E47885F6C21090000FE0FF64C0
:1054E500016005EF64037010D2307F01122ECA7F70
:1054F500401255237F01801B90000FE06402701657
:10550500D2307F03122ECA7F05126F1F7F501255AE
:10551500237F03122ECA7F50126F1F7F00221200B5
:1055250016C22F1269EAE4FD7F08124F71C23022BC
:10670300D2127F0A126F1F7F40120016D22F126916
:10671300EAE4FD7F07124F717F03126F607F50120F
:0B6723006F1F30150312557F7F00220E
:106ADD0030000B9000B8E0FF7C0D7DE0800C2000B5
:106AED000E9000B7E0FF7C0D7DC0125C48B2007FB8
:026AFD0019225C
:10614A008F5AE55A24FF922F1269EAE55A70127F94
:10615A0040120016D201E4FD7F09124F71C201807C
:10616A0015E55AB401107F10120016D202E4FD7F21
:0C617A0009124F71C2027F50126F1F22E9
:104DD100C201C202D20C7F50126F1F7F80120016D7
:104DE10075420390000FE0B401163024627F011276
:104DF1000016302407E542D3940050F67F01803538
:104E010090000FE0FF64026005EF640370413024FD
:104E1100297F02126F1FD2307F03122ECA7F051223
:104E21000016302407E542D3940050F6C2307F02C9
:104E3100122ECA7F05126F1F80153025127F0212B4
:104E4100001630250AE542D3940040033024F3E5EF
:0D4E51004270907FA0126F1FC20CC21E2283
:03000000026C6F20
:106C6F00758E0078FEE4F6D8FD9000007FFF7E1F42
:0D6C7F00E4F0A3DFFCDEFA758188024C25ED
:10399800C2D530F707B2D563F0FF05F030E70CB2B7
:1039A800D5F4048463F0FF05F080018430D502F477
:0239B8000422E7
:1039BA00EF8DF0A4A8F0CF8CF0A428CE8DF0A42E21
:0239CA00FE22DB
:1039CC00BC000BBE0029EF8DF084FFADF022E4CCDF
:1039DC00F875F008EF2FFFEE33FEEC33FCEE9DECA8
:1039EC00984005FCEE9DFE0FD5F0E9E4CEFD22EDEE
:1039FC00F8F5F0EE8420D21CFEADF075F008EF2F38
:103A0C00FFED33FD4007985006D5F0F222C398FD28
:053A1C000FD5F0EA22C5
:103A2100EB9FF5F0EA9E42F0E99D42F0E89C45F0FB
:013A31002272
:103A32007401FF3395E0FEFDFC080808E6CF2FF67F
:103A420018E6CE3EF618E6CD3DF618E6CC3CF62258
:0C3A5200A42582F582E5F03583F583227F
:103A5E00D083D082F8E4937012740193700DA3A3F7
:103A6E0093F8740193F5828883E47374029368600B
:063A7E00EFA3A3A380DF0B
:106E7600EFC39461400AEF947B5005EF24E0FF22B4
:016E860022E9
:00000001FF
